:020000040000FA
:1000000002EF00F00F013F0E926E000E936E000E95
:10001000946E030E956E0F0E966E000E386F000EE6
:10002000396F000E3A6F000E3B6F000E3C6F806A16
:10003000816A826A836A846A896A8A6A8B6A8C6A3C
:100040008D6A00018B8C006A016A026A036A046A85
:10005000056A066A076A086A096A0A6A0B6A0C6A0C
:100060000D6A0E6A0F6A106A116A126A136A146ABC
:10007000156A166A176A186A196A1A6A1B6A1C6A6C
:100080001D6A1E6A1F6A206A216A226A236A256A1B
:10009000266A276A296A246A286A2A6A2B6A2C6ACD
:1000A0002D6A2E6A2F6A306A316A326A336A346A7C
:1000B000356A366A376A386A396A3A6A3C6A3B6A2C
:1000C0003D6A3E6A3F6A406A416A426A436A446ADC
:1000D000456A466A476A486A496A4A6A4B6A4C6A8C
:1000E0004D6A4E6A506A516A526A536A546A556A36
:1000F000566A576A586A596A5A6A70EC37F070EC57
:1001000037F070EC37F070EC37F02EEC2BF0C00EBF
:100110008A6E8C9C8C9E8C8A8C9A2DEC2CF03F0ED7
:100120008A6E8C9C8C9E8C8A8C9A50EC2CF08B8ADC
:1001300031EC2BF098EC37F0000EAA6E000EA96E91
:10014000A69EA69CA68000000000A850116E000E7E
:10015000AA6E010EA96EA69EA69CA68000000000B5
:10016000A850126E000EAA6E020EA96EA69EA69C44
:10017000A68000000000A850136E000EAA6E030EA9
:10018000A96EA69EA69CA68000000000A850146E32
:10019000000EAA6E040EA96EA69EA69CA680000064
:1001A0000000A850156E000EAA6E050EA96EA69E40
:1001B000A69CA68000000000A850166E000EAA6E35
:1001C000060EA96EA69EA69CA68000000000A85060
:1001D000176E000EAA6E070EA96EA69EA69CA6809C
:1001E00000000000A850186E000EAA6E080EA96E3E
:1001F000A69EA69CA68000000000A850196E000EC6
:10020000AA6E090EA96EA69EA69CA68000000000FC
:10021000A8501A6E000EAA6E0A0EA96EA69EA69C83
:10022000A68000000000A8504C6E6DEC2CF0B2ECE3
:100230002DF01D504E6E4CA423EF01F083A223EF4E
:1002400001F04BEC36F0B2EC2DF080B280B650EFFE
:1002500001F0070E5A5CD8B431EF01F05A2A52EF80
:1002600001F05A6A3EB652EF01F01550380B406E5D
:10027000380E405CD8B441EF01F0080E402643EF41
:1002800001F0000E406E1550C70B156E4050151250
:100290004CB268EC36F06DEC2CF03E8652EF01F07B
:1002A0003E965A6A80B47CEF01F0070E595CD8B4D0
:1002B0005DEF01F0592A7EEF01F0596A3EB47EEFFE
:1002C00001F01550380B406E000E405CD8B46DEF55
:1002D00001F0080E405E6FEF01F0380E406E1550D1
:1002E000C70B156E405015124CB268EC36F06DEC31
:1002F0002CF03E847EEF01F03E94596A4CB446ECFB
:1003000036F080B29EEF01F0070E585CD8B48CEF47
:1003100001F0582AA0EF01F0586A3EB2A0EF01F0B8
:10032000040E415CD8B498EF01F0412A99EF01F036
:10033000416A50EC2CF03E82A0EF01F03E92586AE8
:10034000000E415CD8B4BBEF01F0010E415CD8B4A3
:10035000B0EF0BF0020E415CD8B4E6EF11F0030EE3
:10036000415CD8B421EF21F0040E415CD8B4CDEF4C
:1003700026F023EF01F028EC2BF0410E34EC2BF0AB
:10038000B80E4DEC2BF0700E66EC2BF0100E66ECF8
:100390002BF0100E66EC2BF0100E66EC2BF0000E1E
:1003A00066EC2BF08FEC46F0000E66EC2BF0CFECF9
:1003B00045F0000E66EC2BF0AFEC45F0000E66EC5D
:1003C0002BF0CFEC45F0000E66EC2BF00FEC46F076
:1003D000000E66EC2BF0CFEC46F0000E66EC2BF036
:1003E000CFEC45F0000E66EC2BF08FEC46F0BFEC46
:1003F00048F09FEC46F02BEC2BF0400E34EC2BF049
:10040000B80E4DEC2BF0AFEC46F0000E66EC2BF086
:100410008FEC45F0000E66EC2BF0AFEC46F0000ED2
:1004200066EC2BF0BFEC46F0000E66EC2BF09FEC78
:1004300046F0000E66EC2BF0082A210E085CD8B4BA
:1004400027EF02F0100E66EC2BF01CEF02F0086AAA
:10045000700E66EC2BF028EC2BF0400E34EC2BF0F9
:10046000BA0E4DEC2BF01DA852EF02F0BFEC48F095
:10047000BFEC48F0BFEC48F0BFEC48F0000E66EC73
:100480002BF0BFEC48F0000E66EC2BF0BFEC48F010
:10049000000E66EC2BF0BFEC48F0000E66EC2BF083
:1004A0007CEF02F01BA49EEF02F0FF0E66EC2BF037
:1004B000EFEC47F0FF0E66EC2BF0FFEC47F0FF0E81
:1004C00066EC2BF0FF0E66EC2BF0FF0E66EC2BF0CB
:1004D0003FEC48F0FF0E66EC2BF03FEC47F0FF0ED0
:1004E00066EC2BF0DFEC47F0FF0E66EC2BF03FECF8
:1004F00048F0FF0E66EC2BF0082A1A0E085CD8B400
:1005000087EF02F0000E66EC2BF07CEF02F0086A39
:100510002BEC2BF0400E34EC2BF0BA0E4DEC2BF004
:10052000082A070E085CD8B49BEF02F0000E66ECB8
:100530002BF090EF02F0086A25EF03F0FF0E66EC57
:100540002BF03FEC48F0FF0E66EC2BF03FEC47F051
:10055000FF0E66EC2BF0DFEC47F0FF0E66EC2BF0A5
:100560003FEC48F0FF0E66EC2BF0000E66EC2BF033
:10057000000E66EC2BF01BA2EEEF02F0FF0E66EC15
:100580002BF0FFEC47F0FF0E66EC2BF02FEC48F061
:10059000FF0E66EC2BF09FEC47F0FF0E66EC2BF0A5
:1005A0007FEC47F0FF0E66EC2BF0EFEC47F0FF0E10
:1005B00066EC2BF01FEC47F0FF0E66EC2BF02BECFB
:1005C0002BF0400E34EC2BF0BA0E4DEC2BF0CFECB0
:1005D00047F0FF0E66EC2BF025EF03F0FF0E66EC04
:1005E0002BF03FEC47F0FF0E66EC2BF0FFEC47F0F2
:1005F000FF0E66EC2BF00FEC48F0FF0E66EC2BF0D4
:100600009FEC48F0FF0E66EC2BF0082A0D0E085CFC
:10061000D8B410EF03F0000E66EC2BF005EF03F0FA
:10062000086A2BEC2BF0400E34EC2BF0BA0E4DEC9C
:100630002BF0082A070E085CD8B424EF03F0000E54
:1006400066EC2BF019EF03F0086A2BEC2BF0480E48
:1006500034EC2BF0BA0E4DEC2BF01DB847EF03F045
:100660001BA647EF03F0FF0E66EC2BF00FEC48F0F3
:10067000FF0E66EC2BF02FEC48F0FF0E66EC2BF033
:10068000FFEC47F0FF0E66EC2BF053EF03F0082A67
:10069000140E085CD8B452EF03F0000E66EC2BF099
:1006A00047EF03F0086A2BEC2BF05D0E34EC2BF0D7
:1006B000BA0E4DEC2BF01DB87AEF03F01BB07AEFB9
:1006C00003F0FF0E66EC2BF05FEC47F0FF0E66ECDC
:1006D0002BF0DFEC47F0FF0E66EC2BF00FEC48F050
:1006E000FF0E66EC2BF08FEC47F0FF0E66EC2BF064
:1006F00086EF03F0082A1A0E085CD8B485EF03F0E1
:10070000000E66EC2BF07AEF03F0086A28EC2BF071
:10071000400E34EC2BF0B90E4DEC2BF01DB805EF6C
:1007200005F01CB69FEF03F01CB8CDEF03F01CBA28
:10073000FBEF03F01CBC2BEF04F005EF05F0FF0E00
:1007400066EC2BF04FEC47F0FF0E66EC2BF04FEC15
:1007500048F0FF0E66EC2BF03FEC48F0FF0E66EC25
:100760002BF0FF0E66EC2BF0FF0E3FEC47F0FF0E78
:1007700066EC2BF04FEC47F0FF0E66EC2BF0082AEE
:10078000110E085CD8B4CAEF03F0000E66EC2BF033
:10079000BFEF03F0086A11EF05F0FF0E66EC2BF0D7
:1007A0004FEC47F0FF0E66EC2BF04FEC48F0FF0EDD
:1007B00066EC2BF03FEC48F0FF0E66EC2BF0FF0EE2
:1007C00066EC2BF0FF0ECFEC47F0FF0E66EC2BF043
:1007D0004FEC47F0FF0E66EC2BF0082A110E085C78
:1007E000D8B4F8EF03F0000E66EC2BF0EDEF03F059
:1007F000086A11EF05F0FF0E66EC2BF09FEC47F056
:10080000FF0E66EC2BF05FEC47F0FF0E66EC2BF072
:100810003FEC47F0FF0E66EC2BF0AFEC43F0FF0E21
:1008200066EC2BF05FEC43F0FF0E66EC2BF0DFEC98
:1008300043F0FF0E66EC2BF07FEC43F0FF0E66EC0E
:100840002BF0BFEC43F0FF0E66EC2BF0000E66ECD5
:100850002BF011EF05F0FF0E66EC2BF00FEC48F0DB
:10086000FF0E66EC2BF03FEC47F0FF0E66EC2BF032
:10087000DFEC47F0FF0E66EC2BF0000E66EC2BF081
:100880002B50526E529E010E525CD8B465EF04F0AC
:10089000490E525CD8B48DEF04F0030E525CD8B40C
:1008A000B5EF04F0430E525CD8B4DDEF04F0082A33
:1008B0001E0E085CD8B462EF04F0000E66EC2BF05C
:1008C00057EF04F0086A11EF05F0000E66EC2BF00C
:1008D000FF0E66EC2BF03FEC47F0FF0E66EC2BF0C2
:1008E0004FEC47F0FF0E66EC2BF0BFEC48F0000E2B
:1008F00066EC2BF0BFEC48F0000E66EC2BF0000E1F
:1009000066EC2BF0000E66EC2BF0000E66EC2BF084
:10091000000E66EC2BF011EF05F0000E66EC2BF0EC
:10092000FF0E66EC2BF0DFEC47F0FF0E66EC2BF0D1
:100930004FEC47F0FF0E66EC2BF0BFEC48F0000EDA
:1009400066EC2BF0BFEC48F0000E66EC2BF0000ECE
:1009500066EC2BF0000E66EC2BF0000E66EC2BF034
:10096000000E66EC2BF011EF05F0000E66EC2BF09C
:10097000FF0E66EC2BF04FEC47F0FF0E66EC2BF011
:100980001FEC47F0FF0E66EC2BF04FEC48F0FF0E2B
:1009900066EC2BF0BFEC48F0000E66EC2BF0000E7E
:1009A00066EC2BF0000E66EC2BF0000E66EC2BF0E4
:1009B000000E66EC2BF011EF05F0000E66EC2BF04C
:1009C000FF0E66EC2BF04FEC47F0FF0E66EC2BF0C1
:1009D0003FEC47F0FF0E66EC2BF03FEC47F0FF0ECC
:1009E00066EC2BF0BFEC48F0000E66EC2BF0000E2E
:1009F00066EC2BF0000E66EC2BF0000E66EC2BF094
:100A0000000E66EC2BF011EF05F0082A320E085CA0
:100A1000D8B410EF05F0000E66EC2BF005EF05F0F2
:100A2000086A28EC2BF0730E34EC2BF0B90E4DEC69
:100A30002BF01DB84FEF05F01CA24FEF05F0FF0E95
:100A400066EC2BF03FEC48F0FF0E66EC2BF09FECD1
:100A500047F0FF0E66EC2BF02BEC2BF0400E34EC45
:100A60002BF0B90E4DEC2BF0CFEC47F0FF0E66ECFF
:100A70002BF05FEC47F0FF0E66EC2BF0EFEC47F04D
:100A8000FF0E66EC2BF03FEC47F0FF0E66EC2BF010
:100A90005FEC47F0FF0E66EC2BF06FEF05F0082AD5
:100AA0000E0E085CD8B45AEF05F0000E66EC2BF081
:100AB0004FEF05F0086A2BEC2BF0400E34EC2BF0D6
:100AC000B90E4DEC2BF0082A1F0E085CD8B46EEF5F
:100AD00005F0000E66EC2BF063EF05F0086A2BECD6
:100AE0002BF0600E34EC2BF0B90E4DEC2BF01DB852
:100AF0009FEF05F01CA09FEF05F0FF0E66EC2BF0BA
:100B00008FEC47F0FF0E66EC2BF09FEC47F0FF0EEA
:100B100066EC2BF0FF0E66EC2BF0FF0E66EC2BF074
:100B20006FEC47F0FF0E66EC2BF03FEC48F0FF0E49
:100B300066EC2BF0000E66EC2BF0ABEF05F0082A0C
:100B40001C0E085CD8B4AAEF05F0000E66EC2BF082
:100B50009FEF05F0086A28EC2BF0400E34EC2BF0E8
:100B6000BB0E4DEC2BF04CB0BBEF05F01D504E6EA4
:100B70004F6AD0EF05F01D504E5CD8A43F9A000E8E
:100B80004F5CD8A4C6EF05F01D504E6E3FBAD0EFB3
:100B900005F0000E4E5CD8B4D0EF05F085EC3AF0CD
:100BA000000E4E5CD8A4D9EF05F003EC3BF023EF28
:100BB00006F0400E4E5CD8A4E2EF05F023EC3BF0CB
:100BC00023EF06F0200E4E5CD8A4EBEF05F044ECCA
:100BD0003BF023EF06F0100E4E5CD8A4F4EF05F0C6
:100BE00065EC3BF023EF06F0080E4E5CD8A4FDEF59
:100BF00005F09DEC3BF023EF06F0020E4E5CD8A40E
:100C000006EF06F0EBEC3BF023EF06F0010E4E5C36
:100C1000D8A40FEF06F039EC3CF023EF06F0FF0EFE
:100C200066EC2BF0B9EC3CF04E50B6EC39F0FF0E10
:100C300066EC2BF0FF0E66EC2BF018EC3AF0BFECF4
:100C400048F0BFEC48F028EC2BF0400E34EC2BF0D1
:100C5000BD0E4DEC2BF0000E66EC2BF0DFEC45F0FA
:100C6000000E66EC2BF09FEC46F0000E66EC2BF0CD
:100C7000280E66EC2BF0280E66EC2BF0280E66ECA6
:100C80002BF0280E66EC2BF0280E66EC2BF0000EF5
:100C900066EC2BF028EC2BF0530E34EC2BF0BD0E51
:100CA0004DEC2BF05E0E295CD8A476EF06F0000E1A
:100CB00066EC2BF0BFEC48F0000E66EC2BF0BFECBE
:100CC00048F0000E66EC2BF0000E66EC2BF0000EE8
:100CD00066EC2BF0DFEC42F0000E66EC2BF0CFEC74
:100CE00042F0000E66EC2BF09BEF08F05D0E295CE5
:100CF000D8A49AEF06F0000E66EC2BF0BFEC48F09B
:100D0000000E66EC2BF0BFEC48F0000E66EC2BF00A
:100D1000000E66EC2BF0000E66EC2BF0DFEC42F0E0
:100D2000000E66EC2BF0CFEC42F0000E66EC2BF0E0
:100D30009BEF08F0440E295CD8A4BEEF06F0000E2D
:100D400066EC2BF0BFEC48F0000E66EC2BF0EFECFD
:100D500042F0000E66EC2BF0EFEC42F0000E66EC79
:100D60002BF0400E66EC2BF0000E66EC2BF0BFEC87
:100D700042F0000E66EC2BF09BEF08F0450E295C6C
:100D8000D8A4E2EF06F0000E66EC2BF0BFEC48F0C2
:100D9000000E66EC2BF0EFEC42F0000E66EC2BF050
:100DA000EFEC42F0000E66EC2BF0400E66EC2BF000
:100DB000000E66EC2BF0BFEC42F0000E66EC2BF060
:100DC0009BEF08F03E0E295CD8A406EF07F0000E5A
:100DD00066EC2BF0BFEC48F0000E66EC2BF0BFEC9D
:100DE00048F0000E66EC2BF0000E66EC2BF0000EC7
:100DF00066EC2BF0EFEC42F0000E66EC2BF02FECE3
:100E000043F0000E66EC2BF09BEF08F03F0E295CE0
:100E1000D8A42AEF07F0000E66EC2BF0BFEC48F0E8
:100E2000000E66EC2BF0BFEC48F0000E66EC2BF0E9
:100E3000000E66EC2BF0000E66EC2BF0EFEC42F0AF
:100E4000000E66EC2BF02FEC43F0000E66EC2BF05E
:100E50009BEF08F0220E295CD8A44EEF07F0000E9D
:100E600066EC2BF0BFEC48F0FF0E66EC2BF0CFECFD
:100E700043F0FF0E66EC2BF0CFEC43F0FF0E66EC78
:100E80002BF0BF0E66EC2BF0FF0E66EC2BF06FEC38
:100E900043F0FF0E66EC2BF09BEF08F0230E295C6D
:100EA000D8A472EF07F0000E66EC2BF0BFEC48F010
:100EB000FF0E66EC2BF0CFEC43F0FF0E66EC2BF050
:100EC000CFEC43F0FF0E66EC2BF0BF0E66EC2BF080
:100ED000FF0E66EC2BF06FEC43F0FF0E66EC2BF090
:100EE0009BEF08F01F0E295CD8A496EF07F0000EC8
:100EF00066EC2BF0BFEC48F0000E66EC2BF0BFEC7C
:100F000048F0000E66EC2BF0000E66EC2BF0FF0EA6
:100F100066EC2BF0DFEC43F0FF0E66EC2BF0AFEC51
:100F200043F0FF0E66EC2BF09BEF08F0200E295CDF
:100F3000D8A4BAEF07F0000E66EC2BF0BFEC48F037
:100F4000000E66EC2BF0BFEC48F0000E66EC2BF0C8
:100F5000000E66EC2BF0FF0E66EC2BF0DFEC43F09E
:100F6000FF0E66EC2BF0AFEC43F0FF0E66EC2BF0BF
:100F70009BEF08F0110E295CD8A4DEEF07F0FF0EFE
:100F800066EC2BF05FEC43F0FF0E66EC2BF0BFEC51
:100F900043F0FF0E66EC2BF0AFEC43F0FF0E66EC77
:100FA0002BF0BF0E66EC2BF0FF0E66EC2BF08FECF7
:100FB00043F0FF0E66EC2BF09BEF08F0120E295C5D
:100FC000D8A402EF08F0FF0E66EC2BF05FEC43F0C4
:100FD000FF0E66EC2BF0BFEC43F0FF0E66EC2BF03F
:100FE000AFEC43F0FF0E66EC2BF0BF0E66EC2BF07F
:100FF000FF0E66EC2BF08FEC43F0FF0E66EC2BF04F
:101000009BEF08F0100E295CD8A426EF08F0000E24
:1010100066EC2BF0BFEC48F0000E66EC2BF0000EF7
:1010200066EC2BF0FF0E66EC2BF05FEC43F0FF0E4E
:1010300066EC2BF0DFEC43F0FF0E66EC2BF06FEC70
:1010400043F0FF0E66EC2BF09BEF08F00F0E295CCF
:10105000D8A44AEF08F0000E66EC2BF0BFEC48F085
:10106000000E66EC2BF0000E66EC2BF0FF0E66EC2B
:101070002BF05FEC43F0FF0E66EC2BF0DFEC43F05F
:10108000FF0E66EC2BF06FEC43F0FF0E66EC2BF0DE
:101090009BEF08F0000E66EC2BF0100E66EC2BF0C8
:1010A000100E66EC2BF0100E66EC2BF0100E66ECBA
:1010B0002BF0100E66EC2BF0000E66EC2BF0100EF1
:1010C00066EC2BF0100E66EC2BF0100E66EC2BF09D
:1010D000100E66EC2BF0100E66EC2BF0000E66EC9A
:1010E0002BF0100E66EC2BF0100E66EC2BF0100EB1
:1010F00066EC2BF0100E66EC2BF0100E66EC2BF06D
:10110000000E66EC2BF0400E66EC2BF0000E66EC49
:101110002BF0100E66EC2BF0100E66EC2BF0100E80
:1011200066EC2BF0100E66EC2BF0100E66EC2BF03C
:10113000000E66EC2BF0000E66EC2BF01FEC46F078
:10114000000E66EC2BF0FFEC45F0000E66EC2BF089
:101150000FEC47F0000E66EC2BF028EC2BF0400E65
:1011600034EC2BF0BC0E4DEC2BF0000E66EC2BF0AB
:101170000FEC46F0000E66EC2BF04FEC46F0000E44
:1011800066EC2BF0280E66EC2BF0280E66EC2BF0AC
:10119000280E66EC2BF0280E66EC2BF0280E66EC81
:1011A0002BF0000E66EC2BF028EC2BF0530E34ECF9
:1011B0002BF0BC0E4DEC2BF01550380B406E000E92
:1011C000405CD8A40CEF09F0000E66EC2BF08FEC1D
:1011D00046F0000E66EC2BF0EFEC46F0000E66ECED
:1011E0002BF06FEC46F0000E66EC2BF0AFEC42F00B
:1011F000000E66EC2BF0BFEC48F0000E66EC2BF016
:10120000BFEC48F0000E66EC2BF0BFEC48F0000E8F
:1012100066EC2BF057EF0AF0080E405CD8A439EFCB
:1012200009F0000E66EC2BF08FEC46F0000E66EC39
:101230002BF0EFEC46F0000E66EC2BF06FEC46F076
:10124000000E66EC2BF0BFEC42F0000E66EC2BF0CB
:10125000BFEC48F0000E66EC2BF0BFEC48F0000E3F
:1012600066EC2BF0BFEC48F0000E66EC2BF057EF6D
:101270000AF0100E405CD8A466EF09F0000E66EC90
:101280002BF08FEC46F0000E66EC2BF0EFEC46F006
:10129000000E66EC2BF06FEC46F0000E66EC2BF0C7
:1012A000CFEC42F0000E66EC2BF0BFEC48F0000EE5
:1012B00066EC2BF0BFEC48F0000E66EC2BF0BFECB8
:1012C00048F0000E66EC2BF057EF0AF0180E405C69
:1012D000D8A4AAEF09F0000E66EC2BF0BFEC46F0A4
:1012E000000E66EC2BF09FEC46F0000E66EC2BF047
:1012F0009FEC45F0000E66EC2BF0BFEC48F083A2AB
:1013000096EF09F0FF0E66EC2BF01FEC47F0FF0E96
:1013100066EC2BF03FEC47F0FF0E66EC2BF04FEC49
:1013200048F0FF0E66EC2BF057EF0AF0000E66EC6B
:101330002BF09FEC46F0000E66EC2BF06FEC46F0C5
:10134000000E66EC2BF0BFEC45F0000E66EC2BF0C7
:1013500057EF0AF0200E405CD8A4D7EF09F0000E3A
:1013600066EC2BF08FEC46F0000E66EC2BF0EFEC09
:1013700046F0000E66EC2BF06FEC46F0000E66ECCB
:101380002BF0EFEC42F0000E66EC2BF0BFEC48F0D7
:10139000000E66EC2BF0BFEC48F0000E66EC2BF074
:1013A000BFEC48F0000E66EC2BF057EF0AF0280E69
:1013B000405CD8A404EF0AF0000E66EC2BF08FEC32
:1013C00046F0000E66EC2BF0EFEC46F0000E66ECFB
:1013D0002BF06FEC46F0000E66EC2BF0FFEC42F0C9
:1013E000000E66EC2BF0BFEC48F0000E66EC2BF024
:1013F000BFEC48F0000E66EC2BF0BFEC48F0000E9E
:1014000066EC2BF057EF0AF0300E405CD8A431EFB9
:101410000AF0000E66EC2BF08FEC46F0000E66EC46
:101420002BF0EFEC46F0000E66EC2BF06FEC46F084
:10143000000E66EC2BF00FEC43F0000E66EC2BF088
:10144000BFEC48F0000E66EC2BF0BFEC48F0000E4D
:1014500066EC2BF0BFEC48F0000E66EC2BF057EF7B
:101460000AF0000E66EC2BF08FEC46F0000E66ECF6
:101470002BF0EFEC46F0000E66EC2BF06FEC46F034
:10148000000E66EC2BF01FEC43F0000E66EC2BF028
:10149000BFEC48F0000E66EC2BF0BFEC48F0000EFD
:1014A00066EC2BF0BFEC48F0000E66EC2BF01DA8AC
:1014B00050921DB872EF0AF0020E1F5CD8B47EEF96
:1014C0000AF0030E1F5CD8B47EEF0AF0010E1F5C19
:1014D000D8B47EEF0AF0210E1F5CD8B47EEF0AF07C
:1014E00078EF0AF050B278EF0AF06DEC2CF05082F1
:1014F000206A216A226A236A266A276A2050D4EC6D
:1015000039F028EC2BF0400E34EC2BF0BE0E4DECF5
:101510002BF0080E66EC2BF0F80E66EC2BF0080EA4
:1015200066EC2BF0E00E66EC2BF0200E66EC2BF058
:10153000000E66EC2BF0000E66EC2BF0059CF0EC38
:1015400039F02150D4EC39F028EC2BF05A0E34EC61
:101550002BF0BE0E4DEC2BF0F80E66EC2BF0000ECF
:1015600066EC2BF0E00E66EC2BF0200E66EC2BF018
:10157000E00E66EC2BF0000E66EC2BF0000E66EC35
:101580002BF0059CF0EC39F02250D4EC39F028EC2B
:101590002BF0400E34EC2BF0BF0E4DEC2BF0059CE5
:1015A000F0EC39F0DFEC48F02350D4EC39F028ECC3
:1015B0002BF04E0E34EC2BF0BF0E4DEC2BF0059CB7
:1015C000F0EC39F02650D4EC39F028EC2BF05C0E1E
:1015D00034EC2BF0BF0E4DEC2BF0059CF0EC39F009
:1015E000DFEC48F02750D4EC39F028EC2BF06A0EF1
:1015F00034EC2BF0BF0E4DEC2BF0059CF0EC39F0E9
:101600002BEC2BF0460E34EC2BF0BC0E4DEC2BF0FB
:10161000700E66EC2BF0100E66EC2BF0100E66ECE4
:101620002BF0100E66EC2BF0000E66EC2BF0EFECBE
:1016300045F0000E66EC2BF06FEC46F0000E66EC09
:101640002BF05FEC46F0000E66EC2BF0082A220E21
:10165000085CD8B431EF0BF0100E66EC2BF026EFDF
:101660000BF0086A700E66EC2BF02BEC2BF0460E9C
:1016700034EC2BF0BD0E4DEC2BF0000E66EC2BF095
:10168000AFEC42F0000E66EC2BF0280E66EC2BF06F
:10169000280E66EC2BF0280E66EC2BF0280E66EC7C
:1016A0002BF0280E66EC2BF0000E66EC2BF013509E
:1016B0000F0B406E02EC2FF02BEC2BF0460E34ECAF
:1016C0002BF0BE0E4DEC2BF0000E66EC2BF0BFECB9
:1016D00042F0000E66EC2BF0280E66EC2BF0280E84
:1016E00066EC2BF0280E66EC2BF0280E66EC2BF047
:1016F000280E66EC2BF0000E66EC2BF01450F00B6D
:10170000406E404240424042404202EC2FF02BECFF
:101710002BF0460E34EC2BF0BF0E4DEC2BF0000EF0
:1017200066EC2BF0CFEC42F0000E66EC2BF0280EAE
:1017300066EC2BF0280E66EC2BF0280E66EC2BF0F6
:10174000280E66EC2BF0280E66EC2BF0000E66ECF3
:101750002BF014500F0B406E02EC2FF023EF01F032
:101760004F6A28EC2BF0410E34EC2BF0B80E4DEC08
:101770002BF0700E66EC2BF0100E66EC2BF0100EBA
:1017800066EC2BF0100E66EC2BF0000E66EC2BF0E6
:10179000AFEC45F0000E66EC2BF09FEC46F0000E2F
:1017A00066EC2BF02FEC43F0000E66EC2BF0EFEC28
:1017B00042F0000E66EC2BF0BFEC42F0000E66EC3F
:1017C0002BF00FEC43F0000E66EC2BF0BFEC48F072
:1017D0008FEC46F0000E66EC2BF0CFEC45F0000EDF
:1017E00066EC2BF0EFEC45F02BEC2BF0400E34ECDC
:1017F0002BF0B80E4DEC2BF0000E66EC2BF00FEC3E
:1018000046F0000E66EC2BF09FEC46F0000E66EC06
:101810002BF0AFEC46F0000E66EC2BF0CFEC45F071
:10182000000E66EC2BF08FEC46F0000E66EC2BF011
:10183000082A200E085CD8B423EF0CF0100E66ECDA
:101840002BF018EF0CF0086A700E66EC2BF028EC09
:101850002BF0410E34EC2BF0B90E4DEC2BF0FF0EBB
:1018600066EC2BF01FEC47F0FF0E66EC2BF04FEC14
:1018700047F0FF0E66EC2BF04FEC47F0FF0E66ECE6
:101880002BF02FEC48F0FF0E66EC2BF05FEC47F0EE
:10189000FF0E66EC2BF03FEC48F0FF0E66EC2BF0F1
:1018A0003FEC48F0FF0E66EC2BF02BEC2BF0410EDA
:1018B00034EC2BF0B90E4DEC2BF0FF0E66EC2BF058
:1018C0004FEC47F0FF0E66EC2BF01FEC47F0FF0EDD
:1018D00066EC2BF04FEC48F0FF0E66EC2BF01FECA3
:1018E00047F0FF0E66EC2BF080B091EF0CF0070E86
:1018F000555CD8B47FEF0CF0552A93EF0CF0556A85
:101900003EB093EF0CF0060E425CD8B48BEF0CF0B7
:10191000422A8CEF0CF0426A50EC2CF03E8093EFA0
:101920000CF03E90556A84B6B1EF0CF0070E545C93
:10193000D8B49EEF0CF0542AB3EF0CF0546A3EBCBE
:10194000B3EF0CF0000E425CD8B4AAEF0CF04206E4
:10195000ACEF0CF0060E426E50EC2CF03E8CB3EF68
:101960000CF03E9C546A28EC2BF0410E34EC2BF02A
:10197000BA0E4DEC2BF0000E425CD8B4E0EF0CF048
:10198000010E425CD8B4A6EF0DF0020E425CD8B452
:101990006CEF0EF0030E425CD8B432EF0FF0040E81
:1019A000425CD8B4F8EF0FF0050E425CD8B4BEEF3D
:1019B00010F0060E425CD8B484EF11F0E2EF11F0A3
:1019C000AFEC42F0000E66EC2BF0AFEC42F0000EF4
:1019D00066EC2BF0FFEC45F0000E66EC2BF02BECE8
:1019E0002BF0410E34EC2BF0BA0E4DEC2BF01150D5
:1019F0002EEC3AF028EC2BF0410E34EC2BF0BB0E21
:101A00004DEC2BF0AFEC42F0000E66EC2BF0BFEC8F
:101A100042F0000E66EC2BF0FFEC45F0000E66EC99
:101A20002BF02BEC2BF0410E34EC2BF0BB0E4DECDD
:101A30002BF012502EEC3AF028EC2BF0410E34EC47
:101A40002BF0BC0E4DEC2BF0AFEC42F0000E66EC30
:101A50002BF0CFEC42F0000E66EC2BF0FFEC45F0E3
:101A6000000E66EC2BF02BEC2BF0410E34EC2BF03F
:101A7000BC0E4DEC2BF013502EEC3AF028EC2BF072
:101A8000410E34EC2BF0BD0E4DEC2BF0AFEC42F0E0
:101A9000000E66EC2BF0DFEC42F0000E66EC2BF053
:101AA000FFEC45F0000E66EC2BF02BEC2BF0410E1A
:101AB00034EC2BF0BD0E4DEC2BF014502EEC3AF024
:101AC00028EC2BF0410E34EC2BF0BE0E4DEC2BF03D
:101AD000AFEC42F0000E66EC2BF0EFEC42F0000EA3
:101AE00066EC2BF0FFEC45F0000E66EC2BF02BECD7
:101AF0002BF0410E34EC2BF0BE0E4DEC2BF01550BC
:101B00002EEC3AF028EC2BF0410E34EC2BF0BF0E0B
:101B10004DEC2BF0AFEC42F0000E66EC2BF0FFEC3E
:101B200042F0000E66EC2BF0FFEC45F0000E66EC88
:101B30002BF02BEC2BF0410E34EC2BF0BF0E4DECC8
:101B40002BF016502EEC3AF0E2EF11F0AFEC42F031
:101B5000000E66EC2BF00FEC43F0000E66EC2BF061
:101B6000FFEC45F0000E66EC2BF02BEC2BF0410E59
:101B700034EC2BF0BA0E4DEC2BF017502EEC3AF063
:101B800028EC2BF0410E34EC2BF0BB0E4DEC2BF07F
:101B9000AFEC42F0000E66EC2BF01FEC43F0000EB1
:101BA00066EC2BF0FFEC45F0000E66EC2BF02BEC16
:101BB0002BF0410E34EC2BF0BB0E4DEC2BF01850FB
:101BC0002EEC3AF028EC2BF0410E34EC2BF0BC0E4E
:101BD0004DEC2BF0AFEC42F0000E66EC2BF02FEC4E
:101BE00043F0000E66EC2BF0FFEC45F0000E66ECC7
:101BF0002BF02BEC2BF0410E34EC2BF0BC0E4DEC0B
:101C00002BF019502EEC3AF028EC2BF0410E34EC6E
:101C10002BF0BD0E4DEC2BF0AFEC42F0000E66EC5D
:101C20002BF03FEC43F0000E66EC2BF0FFEC45F0A0
:101C3000000E66EC2BF02BEC2BF0410E34EC2BF06D
:101C4000BD0E4DEC2BF01A502EEC3AF028EC2BF098
:101C5000410E34EC2BF0BE0E4DEC2BF0AFEC42F00D
:101C6000000E66EC2BF08FEC45F0000E66EC2BF0CE
:101C7000FFEC45F0000E66EC2BF02BEC2BF0410E48
:101C800034EC2BF0BE0E4DEC2BF01B502EEC3AF04A
:101C900028EC2BF0410E34EC2BF0BF0E4DEC2BF06A
:101CA000AFEC42F0000E66EC2BF09FEC45F0000E1E
:101CB00066EC2BF0FFEC45F0000E66EC2BF02BEC05
:101CC0002BF0410E34EC2BF0BF0E4DEC2BF01C50E2
:101CD0002EEC3AF0E2EF11F0AFEC42F0000E66ECC1
:101CE0002BF0AFEC45F0000E66EC2BF0FFEC45F06E
:101CF000000E66EC2BF02BEC2BF0410E34EC2BF0AD
:101D0000BA0E4DEC2BF01D502EEC3AF028EC2BF0D7
:101D1000410E34EC2BF0BB0E4DEC2BF0AFEC42F04F
:101D2000000E66EC2BF0BFEC45F0000E66EC2BF0DD
:101D3000FFEC45F0000E66EC2BF02BEC2BF0410E87
:101D400034EC2BF0BB0E4DEC2BF01E502EEC3AF089
:101D500028EC2BF0410E34EC2BF0BC0E4DEC2BF0AC
:101D6000AFEC42F0000E66EC2BF0CFEC45F0000E2D
:101D700066EC2BF0FFEC45F0000E66EC2BF02BEC44
:101D80002BF0410E34EC2BF0BC0E4DEC2BF01F5021
:101D90002EEC3AF028EC2BF0410E34EC2BF0BD0E7B
:101DA0004DEC2BF0AFEC42F0000E66EC2BF0DFECCC
:101DB00045F0000E66EC2BF0FFEC45F0000E66ECF3
:101DC0002BF02BEC2BF0410E34EC2BF0BD0E4DEC38
:101DD0002BF020502EEC3AF028EC2BF0410E34EC96
:101DE0002BF0BE0E4DEC2BF0BFEC42F0000E66EC7B
:101DF0002BF0AFEC42F0000E66EC2BF0FFEC45F060
:101E0000000E66EC2BF02BEC2BF0410E34EC2BF09B
:101E1000BE0E4DEC2BF021502EEC3AF028EC2BF0BE
:101E2000410E34EC2BF0BF0E4DEC2BF0BFEC42F02A
:101E3000000E66EC2BF0BFEC42F0000E66EC2BF0CF
:101E4000FFEC45F0000E66EC2BF02BEC2BF0410E76
:101E500034EC2BF0BF0E4DEC2BF022502EEC3AF070
:101E6000E2EF11F0BFEC42F0000E66EC2BF0CFEC8D
:101E700042F0000E66EC2BF0FFEC45F0000E66EC35
:101E80002BF02BEC2BF0410E34EC2BF0BA0E4DEC7A
:101E90002BF023502EEC3AF028EC2BF0410E34ECD2
:101EA0002BF0BB0E4DEC2BF0BFEC42F0000E66ECBD
:101EB0002BF0DFEC42F0000E66EC2BF0FFEC45F06F
:101EC000000E66EC2BF02BEC2BF0410E34EC2BF0DB
:101ED000BB0E4DEC2BF024502EEC3AF028EC2BF0FE
:101EE000410E34EC2BF0BC0E4DEC2BF0BFEC42F06D
:101EF000000E66EC2BF0EFEC42F0000E66EC2BF0DF
:101F0000FFEC45F0000E66EC2BF02BEC2BF0410EB5
:101F100034EC2BF0BC0E4DEC2BF025502EEC3AF0AF
:101F200028EC2BF0410E34EC2BF0BD0E4DEC2BF0D9
:101F3000BFEC42F0000E66EC2BF0FFEC42F0000E1E
:101F400066EC2BF0FFEC45F0000E66EC2BF02BEC72
:101F50002BF0410E34EC2BF0BD0E4DEC2BF0265047
:101F60002EEC3AF028EC2BF0410E34EC2BF0BE0EA8
:101F70004DEC2BF0BFEC42F0000E66EC2BF00FECBA
:101F800043F0000E66EC2BF0FFEC45F0000E66EC23
:101F90002BF02BEC2BF0410E34EC2BF0BE0E4DEC65
:101FA0002BF027502EEC3AF028EC2BF0410E34ECBD
:101FB0002BF0BF0E4DEC2BF0BFEC42F0000E66ECA8
:101FC0002BF01FEC43F0000E66EC2BF0FFEC45F01D
:101FD000000E66EC2BF02BEC2BF0410E34EC2BF0CA
:101FE000BF0E4DEC2BF028502EEC3AF0E2EF11F042
:101FF000BFEC42F0000E66EC2BF02FEC43F0000E2D
:1020000066EC2BF0FFEC45F0000E66EC2BF02BECB1
:102010002BF0410E34EC2BF0BA0E4DEC2BF0295086
:102020002EEC3AF028EC2BF0410E34EC2BF0BB0EEA
:102030004DEC2BF0BFEC42F0000E66EC2BF03FECC9
:1020400043F0000E66EC2BF0FFEC45F0000E66EC62
:102050002BF02BEC2BF0410E34EC2BF0BB0E4DECA7
:102060002BF02A502EEC3AF028EC2BF0410E34ECF9
:102070002BF0BC0E4DEC2BF0BFEC42F0000E66ECEA
:102080002BF08FEC45F0000E66EC2BF0FFEC45F0EA
:10209000000E66EC2BF02BEC2BF0410E34EC2BF009
:1020A000BC0E4DEC2BF02B502EEC3AF028EC2BF024
:1020B000410E34EC2BF0BD0E4DEC2BF0BFEC42F09A
:1020C000000E66EC2BF09FEC45F0000E66EC2BF05A
:1020D000FFEC45F0000E66EC2BF02BEC2BF0410EE4
:1020E00034EC2BF0BD0E4DEC2BF02C502EEC3AF0D6
:1020F00028EC2BF0410E34EC2BF0BE0E4DEC2BF007
:10210000BFEC42F0000E66EC2BF0AFEC45F0000E99
:1021100066EC2BF0FFEC45F0000E66EC2BF02BECA0
:102120002BF0410E34EC2BF0BE0E4DEC2BF02D506D
:102130002EEC3AF028EC2BF0410E34EC2BF0BF0ED5
:102140004DEC2BF0BFEC42F0000E66EC2BF0BFEC38
:1021500045F0000E66EC2BF0FFEC45F0000E66EC4F
:102160002BF02BEC2BF0410E34EC2BF0BF0E4DEC92
:102170002BF02E502EEC3AF0E2EF11F0BFEC42F0D3
:10218000000E66EC2BF0CFEC45F0000E66EC2BF069
:10219000FFEC45F0000E66EC2BF02BEC2BF0410E23
:1021A00034EC2BF0BA0E4DEC2BF02F502EEC3AF015
:1021B00028EC2BF0410E34EC2BF0BB0E4DEC2BF049
:1021C000BFEC42F0000E66EC2BF0DFEC45F0000EA9
:1021D00066EC2BF0FFEC45F0000E66EC2BF02BECE0
:1021E0002BF0410E34EC2BF0BB0E4DEC2BF03050AD
:1021F0002EEC3AF028EC2BF0410E34EC2BF0BC0E18
:102200004DEC2BF0CFEC42F0000E66EC2BF0AFEC77
:1022100042F0000E66EC2BF0FFEC45F0000E66EC91
:102220002BF02BEC2BF0410E34EC2BF0BC0E4DECD4
:102230002BF031502EEC3AF028EC2BF0410E34EC20
:102240002BF0BD0E4DEC2BF0CFEC42F0000E66EC07
:102250002BF0BFEC42F0000E66EC2BF0FFEC45F0EB
:10226000000E66EC2BF02BEC2BF0410E34EC2BF037
:10227000BD0E4DEC2BF032502EEC3AF028EC2BF04A
:10228000410E34EC2BF0BE0E4DEC2BF0CFEC42F0B7
:10229000000E66EC2BF0CFEC42F0000E66EC2BF05B
:1022A000FFEC45F0000E66EC2BF02BEC2BF0410E12
:1022B00034EC2BF0BE0E4DEC2BF033502EEC3AF0FC
:1022C00028EC2BF0410E34EC2BF0BF0E4DEC2BF034
:1022D000CFEC42F0000E66EC2BF0DFEC42F0000E8B
:1022E00066EC2BF0FFEC45F0000E66EC2BF02BECCF
:1022F0002BF0410E34EC2BF0BF0E4DEC2BF0345094
:102300002EEC3AF0E2EF11F0CFEC42F0000E66EC6A
:102310002BF0EFEC42F0000E66EC2BF0FFEC45F0FA
:10232000000E66EC2BF02BEC2BF0410E34EC2BF076
:10233000BA0E4DEC2BF035502EEC3AF028EC2BF089
:10234000410E34EC2BF0BB0E4DEC2BF0CFEC42F0F9
:10235000000E66EC2BF0FFEC42F0000E66EC2BF06A
:10236000FFEC45F0000E66EC2BF02BEC2BF0410E51
:1023700034EC2BF0BB0E4DEC2BF036502EEC3AF03B
:1023800028EC2BF0410E34EC2BF0BC0E4DEC2BF076
:10239000CFEC42F0000E66EC2BF00FEC43F0000E99
:1023A00066EC2BF0FFEC45F0000E66EC2BF02BEC0E
:1023B0002BF0410E34EC2BF0BC0E4DEC2BF03750D3
:1023C0002EEC3AF0E9EC2EF023EF01F028EC2BF0A4
:1023D000410E34EC2BF0B80E4DEC2BF0700E66EC89
:1023E0002BF0100E66EC2BF0100E66EC2BF0100E9E
:1023F00066EC2BF0000E66EC2BF0AFEC45F0000E17
:1024000066EC2BF09FEC46F0000E66EC2BF02FEC08
:1024100043F0000E66EC2BF0EFEC42F0000E66ECA1
:102420002BF0BFEC42F0000E66EC2BF00FEC43F00B
:10243000000E66EC2BF0BFEC48F09FEC46F0000E6F
:1024400066EC2BF0CFEC45F0000E66EC2BF0AFEC19
:1024500046F02BEC2BF0400E34EC2BF0B80E4DEC8C
:102460002BF0000E66EC2BF0AFEC46F0000E66ECA5
:102470002BF00FEC46F0000E66EC2BF04FEC46F024
:10248000000E66EC2BF0EFEC45F0000E66EC2BF046
:10249000082A260E085CD8B453EF12F0100E66EC32
:1024A0002BF048EF12F0086A700E66EC2BF0000E6D
:1024B000435CD8B463EF12F0010E435CD8B4A3EFD1
:1024C00015F023EF01F028EC2BF0460E34EC2BF046
:1024D000B90E4DEC2BF09FEC46F0000E66EC2BF0A5
:1024E000CFEC45F0000E66EC2BF02FEC46F0000E22
:1024F00066EC2BF0CFEC45F0000E66EC2BF0AFEC69
:1025000045F0000E66EC2BF0AFEC46F0000E66ECEA
:102510002BF0BFEC48F08FEC45F0000E66EC2BF092
:10252000BFEC45F0000E66EC2BF0BFEC45F02BEC59
:102530002BF0400E34EC2BF0B90E4DEC2BF0000ECE
:1025400066EC2BF08FEC46F0000E66EC2BF0CFEC37
:1025500045F0000E66EC2BF09FEC46F0000E66ECAA
:102560002BF09FEC46F0000E66EC2BF080B0D1EF24
:1025700012F0070E555CD8B4C1EF12F0552AD3EF14
:1025800012F0556A3EB0D3EF12F00A0E465CD8B492
:10259000CDEF12F0462ACEEF12F0466A3E80D3EF1E
:1025A00012F03E90556A84B6EFEF12F0070E545CBD
:1025B000D8B4DEEF12F0542AF1EF12F0546A3EBCA8
:1025C000F1EF12F0000E465CD8B4EAEF12F04606C6
:1025D000ECEF12F00A0E466E3E8CF1EF12F03E9CCC
:1025E000546A3F9428EC2BF04A0E34EC2BF0BB0ECF
:1025F0004DEC2BF0000E465CD8B413EF13F0000E38
:1026000066EC2BF0AFEC42F0000E66EC2BF0AFEC7A
:1026100042F0000E66EC2BF0FFEC45F0000E66EC8D
:102620002BF025EF13F0FF0E66EC2BF04FEC43F090
:10263000FF0E66EC2BF04FEC43F0FF0E66EC2BF038
:102640008FEC47F0FF0E66EC2BF028EC2BF0670EBA
:1026500034EC2BF0BB0E4DEC2BF0010E465CD8B4E5
:1026600046EF13F0000E66EC2BF0AFEC42F0000EDC
:1026700066EC2BF0BFEC42F0000E66EC2BF0FFECAA
:1026800045F0000E66EC2BF058EF13F0FF0E66ECF1
:102690002BF04FEC43F0FF0E66EC2BF05FEC43F0B9
:1026A000FF0E66EC2BF08FEC47F0FF0E66EC2BF084
:1026B0002BEC2BF0440E34EC2BF0BB0E4DEC2BF03E
:1026C000020E465CD8B479EF13F0000E66EC2BF0E6
:1026D000AFEC42F0000E66EC2BF0CFEC42F0000EB7
:1026E00066EC2BF0FFEC45F0000E66EC2BF08BEF68
:1026F00013F0FF0E66EC2BF04FEC43F0FF0E66EC90
:102700002BF06FEC43F0FF0E66EC2BF08FEC47F0F4
:10271000FF0E66EC2BF02BEC2BF0610E34EC2BF063
:10272000BB0E4DEC2BF0030E465CD8B4ACEF13F0AF
:10273000000E66EC2BF0AFEC42F0000E66EC2BF0D6
:10274000DFEC42F0000E66EC2BF0FFEC45F0000EE3
:1027500066EC2BF0BEEF13F0FF0E66EC2BF04FECA7
:1027600043F0FF0E66EC2BF07FEC43F0FF0E66ECBF
:102770002BF08FEC47F0FF0E66EC2BF028EC2BF0E3
:102780004A0E34EC2BF0BC0E4DEC2BF0040E465CE4
:10279000D8B4DFEF13F0000E66EC2BF0AFEC42F094
:1027A000000E66EC2BF0EFEC42F0000E66EC2BF026
:1027B000FFEC45F0000E66EC2BF0F1EF13F0FF0E8E
:1027C00066EC2BF04FEC43F0FF0E66EC2BF08FEC39
:1027D00043F0FF0E66EC2BF08FEC47F0FF0E66EC3B
:1027E0002BF028EC2BF0670E34EC2BF0BC0E4DECEC
:1027F0002BF0050E465CD8B412EF14F0000E66EC18
:102800002BF0AFEC42F0000E66EC2BF0FFEC42F048
:10281000000E66EC2BF0FFEC45F0000E66EC2BF0A2
:1028200024EF14F0FF0E66EC2BF04FEC43F0FF0E9C
:1028300066EC2BF09FEC43F0FF0E66EC2BF08FEC78
:1028400047F0FF0E66EC2BF02BEC2BF0440E34EC33
:102850002BF0BC0E4DEC2BF0060E465CD8B445EFC9
:1028600014F0000E66EC2BF0AFEC42F0000E66ECBC
:102870002BF00FEC43F0000E66EC2BF0FFEC45F074
:10288000000E66EC2BF057EF14F0FF0E66EC2BF009
:102890004FEC43F0FF0E66EC2BF0AFEC43F0FF0E75
:1028A00066EC2BF08FEC47F0FF0E66EC2BF02BEC78
:1028B0002BF0610E34EC2BF0B40E4DEC2BF0070E28
:1028C000465CD8B478EF14F0000E66EC2BF0AFEC59
:1028D00042F0000E66EC2BF01FEC43F0000E66ECAD
:1028E0002BF0FFEC45F0000E66EC2BF08AEF14F0B5
:1028F000FF0E66EC2BF04FEC43F0FF0E66EC2BF076
:10290000BFEC43F0FF0E66EC2BF08FEC47F0FF0EB0
:1029100066EC2BF028EC2BF04A0E34EC2BF0BD0EBD
:102920004DEC2BF0080E465CD8B4ABEF14F0000E63
:1029300066EC2BF0AFEC42F0000E66EC2BF02FECC7
:1029400043F0000E66EC2BF0FFEC45F0000E66EC59
:102950002BF0BDEF14F0FF0E66EC2BF04FEC43F0C4
:10296000FF0E66EC2BF0CFEC43F0FF0E66EC2BF085
:102970008FEC47F0FF0E66EC2BF028EC2BF0670E87
:1029800034EC2BF0BD0E4DEC2BF0090E465CD8B4A8
:10299000DEEF14F0000E66EC2BF0AFEC42F0000E10
:1029A00066EC2BF03FEC43F0000E66EC2BF0FFECF6
:1029B00045F0000E66EC2BF0F0EF14F0FF0E66EC25
:1029C0002BF04FEC43F0FF0E66EC2BF0DFEC43F006
:1029D000FF0E66EC2BF08FEC47F0FF0E66EC2BF051
:1029E00028EC2BF04A0E34EC2BF0BF0E4DEC2BF004
:1029F0000A0E465CD8B443EF15F0000E66EC2BF0DF
:102A0000BFEC45F0000E66EC2BF0CFEC45F0000E6D
:102A100066EC2BF0DFEC45F0000E66EC2BF08FEC53
:102A200045F0000E66EC2BF0BFEC46F0000E66ECB5
:102A30002BF02FEC46F0000E66EC2BF0AFEC46F0DE
:102A4000000E66EC2BF0BFEC48F02FEC46F0000EC9
:102A500066EC2BF02BEC2BF0400E34EC2BF0BF0E81
:102A60004DEC2BF05FEC46F0000E66EC2BF08FEC9B
:102A700045F0000E66EC2BF0BFEC45F0000E66EC66
:102A80002BF087EF15F0FF0E66EC2BF04FEC47F0C4
:102A9000FF0E66EC2BF05FEC47F0FF0E66EC2BF0C0
:102AA0006FEC47F0FF0E66EC2BF01FEC47F0FF0ECB
:102AB00066EC2BF05FEC48F0FF0E66EC2BF0CFECF1
:102AC00047F0FF0E66EC2BF04FEC48F0FF0E66EC83
:102AD0002BF0CFEC48F0CFEC47F0FF0E66EC2BF07C
:102AE0002BEC2BF0400E34EC2BF0BF0E4DEC2BF00A
:102AF000FFEC47F0FF0E66EC2BF01FEC47F0FF0EEB
:102B000066EC2BF04FEC47F0FF0E66EC2BF0E9EC97
:102B10002EF080B89FEF15F0070E575CD8B494EFF5
:102B200015F0572AA1EF15F0576A3EB8A1EF15F03E
:102B3000010E436E50EC2CF03E88A1EF15F03E984C
:102B4000576A23EF01F028EC2BF0460E34EC2BF003
:102B5000B90E4DEC2BF0000E465CD8B4DFEF15F04B
:102B6000010E465CD8B4E0EF16F0020E465CD8B415
:102B700039EF18F0030E465CD8B44DEF19F0040E8F
:102B8000465CD8B431EF1AF0050E465CD8B440EF7D
:102B90001BF0060E465CD8B467EF1CF0070E465CCF
:102BA000D8B4CBEF1DF0080E465CD8B483EF1EF00E
:102BB000090E465CD8B43BEF1FF0F3EF1FF0FCECBE
:102BC0003CF03FB2E6EF15F0050E496E3FB449EF19
:102BD00016F080B017EF16F0070E555CD8B4F4EF7E
:102BE00015F0552A19EF16F0556A3EB019EF16F098
:102BF000010E495CD8A401EF16F0080E496E14EFDF
:102C000016F0040E495CD8A40AEF16F0010E496EC6
:102C100014EF16F0080E495CD8A413EF16F0050E59
:102C2000496E14EF16F049063E8019EF16F03E90FB
:102C3000556A84B647EF16F0070E545CD8B424EFFB
:102C400016F0542A49EF16F0546A3EBC49EF16F0CC
:102C5000080E495CD8A431EF16F0010E496E44EF1E
:102C600016F0010E495CD8A43AEF16F0040E496E36
:102C700044EF16F0050E495CD8A443EF16F0080E99
:102C8000496E44EF16F0492A3E8C49EF16F03E9CFF
:102C9000546A28EC2BF0460E34EC2BF0BC0E4DECB5
:102CA0002BF0010E495CD8B483EF16F0040E495C9A
:102CB000D8B4A6EF16F0080E495CD8B4C7EF16F0EA
:102CC000FF0E66EC2BF04FEC48F0FF0E66EC2BF09D
:102CD0002FEC48F0FF0E66EC2BF05FEC48F0FF0E97
:102CE00066EC2BF0EFEC47F0FF0E66EC2BF03FECC0
:102CF00047F0FF0E66EC2BF0BFEC48F0000E66ECE0
:102D00002BF0C7EF16F0FF0E66EC2BF06FEC47F0E0
:102D1000FF0E66EC2BF03FEC48F0FF0E66EC2BF05C
:102D20007FEC48F0FF0E66EC2BF03FEC47F0FF0E17
:102D300066EC2BF0CFEC47F0FF0E66EC2BF0BFEC0F
:102D400047F0FF0E66EC2BF0C7EF16F0FF0E66ECB7
:102D50002BF00FEC48F0FF0E66EC2BF04FEC47F039
:102D6000FF0E66EC2BF05FEC48F0FF0E66EC2BF0EC
:102D70002FEC48F0FF0E66EC2BF0BFEC48F0000E95
:102D800066EC2BF0BFEC48F0000E66EC2BF03FB683
:102D9000CEEF16F03F8611504A6E4B6E97EC32F034
:102DA0002BEC2BF0400E34EC2BF0BD0E4DEC2BF049
:102DB000405046EC3AF08FEC3AF03F82FEEF20F0C4
:102DC00055EC3DF03FB2E7EF16F0070E496E3FA419
:102DD0001DEC32F028EC2BF0460E34EC2BF0BC0E40
:102DE0004DEC2BF0000E495CD8B442EF17F0010E09
:102DF000495CD8B46AEF17F0020E495CD8B492EF80
:102E000017F0030E495CD8B492EF17F0040E495C3A
:102E1000D8B4C6EF17F0050E495CD8B4C6EF17F06A
:102E2000060E495CD8B4FAEF17F0080E495CD8B426
:102E300020EF18F0FF0E66EC2BF03FEC47F0FF0E92
:102E400066EC2BF08FEC47F0FF0E66EC2BF03FECBE
:102E500048F0FF0E66EC2BF0BFEC48F0000E66EC7D
:102E60002BF0BFEC48F0000E66EC2BF0BFEC48F006
:102E7000000E66EC2BF0BFEC48F0000E66EC2BF079
:102E800020EF18F0FF0E66EC2BF03FEC48F0FF0E41
:102E900066EC2BF07FEC48F0FF0E66EC2BF03FEC7D
:102EA00047F0FF0E66EC2BF0CFEC47F0FF0E66EC20
:102EB0002BF0BFEC47F0FF0E66EC2BF0BFEC48F0B8
:102EC000000E66EC2BF0BFEC48F0000E66EC2BF029
:102ED00020EF18F0FF0E66EC2BF0DFEC47F0FF0E52
:102EE00066EC2BF05FEC48F0FF0E66EC2BF04FEC3D
:102EF00048F0FF0E66EC2BF05FEC47F0FF0E66EC3F
:102F00002BF03FEC48F0FF0E66EC2BF01FEC47F087
:102F1000FF0E66EC2BF0FFEC47F0FF0E66EC2BF09B
:102F200020EF18F0FF0E66EC2BF09FEC47F0FF0E41
:102F300066EC2BF0EFEC47F0FF0E66EC2BF04FEC5D
:102F400048F0FF0E66EC2BF0020E495CD8B4B0EFEF
:102F500017F04FEC43F0FF0E66EC2BF0B5EF17F0D7
:102F60005FEC43F0FF0E66EC2BF0BFEC48F0000E78
:102F700066EC2BF0BFEC48F0000E66EC2BF0BFECDB
:102F800048F0000E66EC2BF020EF18F0FF0E66EC18
:102F90002BF08FEC47F0FF0E66EC2BF0FFEC47F0C8
:102FA000FF0E66EC2BF0CFEC47F0FF0E66EC2BF03B
:102FB0004FEC47F0FF0E66EC2BF0040E495CD8B4E2
:102FC000E9EF17F04FEC43F0FF0E66EC2BF0EEEF5D
:102FD00017F05FEC43F0FF0E66EC2BF0BFEC48F00F
:102FE000000E66EC2BF0BFEC48F0000E66EC2BF008
:102FF00020EF18F0FF0E66EC2BF02FEC48F0FF0EE0
:1030000066EC2BF0DFEC47F0FF0E66EC2BF03FECAC
:1030100047F0FF0E66EC2BF0BFEC47F0FF0E66ECBE
:103020002BF06FEC47F0FF0E66EC2BF0BFEC48F096
:10303000000E66EC2BF0BFEC48F0000E66EC2BF0B7
:103040003FB627EF18F03F8612504A6E4B6E97EC52
:1030500032F02BEC2BF0400E34EC2BF0BD0E4DEC8F
:103060002BF0405046EC3AF08FEC3AF03F82FEEF06
:1030700020F0AEEC3DF03FB240EF18F0070E496E85
:103080003FA41DEC32F028EC2BF0460E34EC2BF074
:10309000BC0E4DEC2BF0000E495CD8B4BAEF18F022
:1030A000010E495CD8B4ECEF18F0020E495CD8B4BC
:1030B000ECEF18F0030E495CD8B4ECEF18F0080EF2
:1030C000495CD8B434EF19F0FF0E66EC2BF07FECBE
:1030D00047F0FF0E66EC2BF00FEC48F0FF0E66ECAD
:1030E0002BF0FFEC47F0FF0E66EC2BF04FEC43F0BB
:1030F000FF0E66EC2BF03FEC48F0FF0E66EC2BF079
:103100005FEC47F0FF0E66EC2BF0CFEC47F0FF0EC4
:1031100066EC2BF0040E495CD8B4A0EF18F0050E55
:10312000495CD8B4A7EF18F0060E495CD8B4AEEFEE
:1031300018F04FEC43F0FF0E66EC2BF0B3EF18F0F5
:103140007FEC43F0FF0E66EC2BF0B3EF18F06FEC62
:1031500043F0FF0E66EC2BF0B3EF18F05FEC43F09A
:10316000FF0E66EC2BF0BFEC48F0000E66EC2BF087
:1031700034EF19F0FF0E66EC2BF04FEC47F0FF0E2A
:1031800066EC2BF05FEC47F0FF0E66EC2BF04FEC9B
:1031900048F0FF0E66EC2BF03FEC47F0FF0E66ECBC
:1031A0002BF09FEC47F0FF0E66EC2BF0BFEC48F0E5
:1031B000000E66EC2BF0BFEC48F0000E66EC2BF036
:1031C000BFEC48F0000E66EC2BF0BFEC48F0000EB0
:1031D00066EC2BF034EF19F0FF0E66EC2BF05FEC91
:1031E00047F0FF0E66EC2BF0DFEC47F0FF0E66ECCD
:1031F0002BF00FEC48F0FF0E66EC2BF08FEC47F055
:10320000FF0E66EC2BF03FEC47F0FF0E66EC2BF068
:10321000EFEC47F0FF0E66EC2BF04FEC48F0FF0EA2
:1032200066EC2BF0CFEC47F0FF0E66EC2BF0010EB6
:10323000495CD8B428EF19F0020E495CD8B42FEFDE
:1032400019F04FEC43F0FF0E66EC2BF034EF19F061
:103250006FEC43F0FF0E66EC2BF034EF19F05FECEF
:1032600043F0FF0E66EC2BF03FB63BEF19F03F86C4
:1032700013504A6E4B6E97EC32F02BEC2BF0400E55
:1032800034EC2BF0BD0E4DEC2BF0405046EC3AF0F8
:103290008FEC3AF03F82FEEF20F007EC3EF03FB2B9
:1032A00054EF19F0070E496E3FA41DEC32F028ECE4
:1032B0002BF0460E34EC2BF0BC0E4DEC2BF0000E38
:1032C000495CD8B4C9EF19F0010E495CD8B4C9EF14
:1032D00019F0020E495CD8B4C9EF19F0030E495C2D
:1032E000D8B4C9EF19F0080E495CD8B418EF1AF039
:1032F000FF0E66EC2BF07FEC47F0FF0E66EC2BF038
:103300000FEC48F0FF0E66EC2BF0FFEC47F0FF0EE1
:1033100066EC2BF06FEC43F0FF0E66EC2BF03FEC0D
:1033200048F0FF0E66EC2BF05FEC47F0FF0E66EC0A
:103330002BF0CFEC47F0FF0E66EC2BF0040E495C4F
:10334000D8B4B4EF19F0050E495CD8B4BBEF19F04E
:10335000060E495CD8B4C2EF19F04FEC43F0FF0EF3
:1033600066EC2BF018EF1AF07FEC43F0FF0E66ECE2
:103370002BF018EF1AF06FEC43F0FF0E66EC2BF019
:1033800018EF1AF05FEC43F0FF0E66EC2BF018EF2D
:103390001AF0FF0E66EC2BF07FEC47F0FF0E66ECA8
:1033A0002BF00FEC48F0FF0E66EC2BF0FFEC47F033
:1033B000FF0E66EC2BF05FEC43F0FF0E66EC2BF09B
:1033C0003FEC48F0FF0E66EC2BF05FEC47F0FF0E91
:1033D00066EC2BF0CFEC47F0FF0E66EC2BF0000E06
:1033E000495CD8B405EF1AF0010E495CD8B40CEF73
:1033F0001AF0020E495CD8B413EF1AF04FEC43F008
:10340000FF0E66EC2BF018EF1AF07FEC43F0FF0E86
:1034100066EC2BF018EF1AF06FEC43F0FF0E66EC41
:103420002BF018EF1AF05FEC43F0FF0E66EC2BF078
:103430003FB61FEF1AF03F8614504A6E4B6E97EC62
:1034400032F02BEC2BF0400E34EC2BF0BD0E4DEC9B
:103450002BF0405046EC3AF08FEC3AF03F82FEEF12
:1034600020F060EC3EF03FB238EF1AF0070E496EE4
:103470003FA41DEC32F028EC2BF0460E34EC2BF080
:10348000BC0E4DEC2BF0000E495CD8B46DEF1AF079
:10349000010E495CD8B490EF1AF0020E495CD8B422
:1034A000B3EF1AF0030E495CD8B4B3EF1AF0040E70
:1034B000495CD8B4B3EF1AF0050E495CD8B4EEEF0E
:1034C0001AF0060E495CD8B4EEEF1AF0080E495C0B
:1034D000D8B427EF1BF0EEEF1AF0FF0E66EC2BF0DE
:1034E0002FEC48F0FF0E66EC2BF05FEC48F0FF0E7F
:1034F00066EC2BF0EFEC47F0FF0E66EC2BF0BFEC28
:1035000048F0000E66EC2BF0BFEC48F0000E66ECC5
:103510002BF0BFEC48F0000E66EC2BF027EF1BF011
:10352000FF0E66EC2BF02FEC48F0FF0E66EC2BF054
:103530008FEC48F0FF0E66EC2BF04FEC47F0FF0EDF
:1035400066EC2BF0BFEC48F0000E66EC2BF0BFEC05
:1035500048F0000E66EC2BF0BFEC48F0000E66EC75
:103560002BF027EF1BF0FF0E66EC2BF02FEC48F052
:10357000FF0E66EC2BF08FEC48F0FF0E66EC2BF0A4
:103580003FEC48F0FF0E66EC2BF05FEC47F0FF0ECF
:1035900066EC2BF0CFEC47F0FF0E66EC2BF0020E42
:1035A000495CD8B4E0EF1AF0030E495CD8B4E7EFF9
:1035B0001AF04FEC43F0FF0E66EC2BF027EF1BF0F8
:1035C0006FEC43F0FF0E66EC2BF027EF1BF05FEC87
:1035D00043F0FF0E66EC2BF027EF1BF0FF0E66ECBE
:1035E0002BF04FEC48F0FF0E66EC2BF08FEC48F020
:1035F000FF0E66EC2BF03FEC48F0FF0E66EC2BF074
:103600005FEC47F0FF0E66EC2BF0CFEC47F0FF0EBF
:1036100066EC2BF0050E495CD8B41BEF1BF0060ED0
:10362000495CD8B422EF1BF04FEC43F0FF0E66EC80
:103630002BF027EF1BF06FEC43F0FF0E66EC2BF046
:1036400027EF1BF05FEC43F0FF0E66EC2BF03FB66C
:103650002EEF1BF03F8615504A6E4B6E97EC32F002
:103660002BEC2BF0400E34EC2BF0BD0E4DEC2BF080
:10367000405046EC3AF08FEC3AF03F82FEEF20F0FB
:10368000B9EC3EF03FB247EF1BF0070E496E3FA486
:103690001DEC32F028EC2BF0460E34EC2BF0BC0E77
:1036A0004DEC2BF0080E495CD8B44EEF1CF0FF0E29
:1036B00066EC2BF03FEC48F0FF0E66EC2BF0FFECD5
:1036C00047F0FF0E66EC2BF0000E495CD8B4A2EF79
:1036D0001BF0010E495CD8B4BDEF1BF0020E495C33
:1036E000D8B4D8EF1BF0030E495CD8B4D8EF1BF068
:1036F000040E495CD8B4FFEF1BF0050E495CD8B44A
:103700001AEF1CF0060E495CD8B435EF1CF0CFEC74
:1037100047F0FF0E66EC2BF02FEC48F0FF0E66EC46
:103720002BF00FEC48F0FF0E66EC2BF0FFEC47F0AF
:10373000FF0E66EC2BF0CFEC47F0FF0E66EC2BF0A3
:103740004EEF1CF0DFEC47F0FF0E66EC2BF03FEC89
:1037500048F0FF0E66EC2BF0BFEC48F0000E66EC74
:103760002BF0BFEC48F0000E66EC2BF0BFEC48F0FD
:10377000000E66EC2BF04EEF1CF03FEC48F0FF0E15
:1037800066EC2BF06FEC47F0FF0E66EC2BF0BFEC15
:1037900048F0000E66EC2BF0BFEC48F0000E66EC33
:1037A0002BF0BFEC48F0000E66EC2BF04EEF1CF057
:1037B0002FEC48F0FF0E66EC2BF05FEC47F0FF0EAD
:1037C00066EC2BF03FEC48F0FF0E66EC2BF0020E9F
:1037D000495CD8B4F3EF1BF04FEC43F0FF0E66ECFE
:1037E0002BF0F8EF1BF05FEC43F0FF0E66EC2BF0D4
:1037F000BFEC48F0000E66EC2BF04EEF1CF0AFEC87
:1038000047F0FF0E66EC2BF05FEC48F0FF0E66EC25
:103810002BF03FEC48F0FF0E66EC2BF04FEC48F03D
:10382000FF0E66EC2BF0BFEC48F0000E66EC2BF0C0
:103830004EEF1CF04FEC47F0FF0E66EC2BF05FEC08
:1038400047F0FF0E66EC2BF0CFEC47F0FF0E66EC76
:103850002BF0BFEC48F0000E66EC2BF0BFEC48F00C
:10386000000E66EC2BF04EEF1CF03FEC48F0FF0E24
:1038700066EC2BF00FEC48F0FF0E66EC2BF0FFEC43
:1038800047F0FF0E66EC2BF0CFEC47F0FF0E66EC36
:103890002BF0BFEC48F0000E66EC2BF03FB655EF76
:1038A0001CF03F8616504A6E4B6E97EC32F02BECB4
:1038B0002BF0400E34EC2BF0BD0E4DEC2BF04050B5
:1038C00046EC3AF08FEC3AF03F82FEEF20F062ECEB
:1038D0003FF03FB26EEF1CF0070E496E3FA45AEC6A
:1038E00032F028EC2BF0460E34EC2BF0BC0E4DECF5
:1038F0002BF0010E495CD8B4C4EF1CF0020E495CF9
:10390000D8B4ECEF1CF0030E495CD8B414EF1DF0F2
:10391000040E495CD8B43CEF1DF0050E495CD8B4E8
:1039200064EF1DF0060E495CD8B48CEF1DF0080E54
:10393000495CD8B4B2EF1DF0FF0E66EC2BF00FEC33
:1039400048F0FF0E66EC2BF01FEC47F0FF0E66EC24
:103950002BF02FEC48F0FF0E66EC2BF0DFEC47F07D
:10396000FF0E66EC2BF0BFEC48F0000E66EC2BF07F
:10397000BFEC48F0000E66EC2BF0BFEC48F0000EF8
:1039800066EC2BF0B2EF1DF0FF0E66EC2BF01FEC97
:1039900048F0FF0E66EC2BF03FEC47F0FF0E66ECB4
:1039A0002BF02FEC48F0FF0E66EC2BF03FEC47F0CD
:1039B000FF0E66EC2BF0DFEC47F0FF0E66EC2BF011
:1039C000BFEC48F0000E66EC2BF0BFEC48F0000EA8
:1039D00066EC2BF0B2EF1DF0FF0E66EC2BF03FEC27
:1039E00047F0FF0E66EC2BF03FEC47F0FF0E66EC65
:1039F0002BF02FEC48F0FF0E66EC2BF03FEC47F07D
:103A0000FF0E66EC2BF0DFEC47F0FF0E66EC2BF0C0
:103A1000BFEC48F0000E66EC2BF0BFEC48F0000E57
:103A200066EC2BF0B2EF1DF0FF0E66EC2BF05FECB6
:103A300048F0FF0E66EC2BF0EFEC47F0FF0E66EC63
:103A40002BF0CFEC47F0FF0E66EC2BF0FFEC47F0CD
:103A5000FF0E66EC2BF03FEC47F0FF0E66EC2BF010
:103A6000BFEC47F0FF0E66EC2BF0DFEC47F0FF0EEB
:103A700066EC2BF0B2EF1DF0FF0E66EC2BF06FEC56
:103A800048F0FF0E66EC2BF0DFEC47F0FF0E66EC23
:103A90002BF0BFEC48F0000E66EC2BF0BFEC48F0CA
:103AA000000E66EC2BF0BFEC48F0000E66EC2BF03D
:103AB000BFEC48F0000E66EC2BF0BFEC48F0000EB7
:103AC00066EC2BF0B2EF1DF0FF0E66EC2BF03FEC36
:103AD00047F0FF0E66EC2BF0FFEC47F0FF0E66ECB4
:103AE0002BF0DFEC47F0FF0E66EC2BF06FEC47F0AD
:103AF000FF0E66EC2BF0DFEC47F0FF0E66EC2BF0D0
:103B0000BFEC48F0000E66EC2BF0BFEC48F0000E66
:103B100066EC2BF0B2EF1DF0FF0E66EC2BF02FECF5
:103B200047F0FF0E66EC2BF09FEC47F0FF0E66ECC3
:103B30002BF00FEC48F0FF0E66EC2BF0DFEC47F0BB
:103B4000FF0E66EC2BF0BFEC48F0000E66EC2BF09D
:103B5000BFEC48F0000E66EC2BF0BFEC48F0000E16
:103B600066EC2BF03FB6B9EF1DF03F8617504A6E5A
:103B70004B6E97EC32F02BEC2BF0400E34EC2BF02C
:103B8000BD0E4DEC2BF0405046EC3AF08FEC3AF085
:103B90003F82FEEF20F0F0EC3FF03FB2D2EF1DF09D
:103BA000070E496E3FA45AEC32F028EC2BF0460E7B
:103BB00034EC2BF0BC0E4DEC2BF0010E495CD8B46C
:103BC00013EF1EF0020E495CD8B421EF1EF0030E75
:103BD000495CD8B42AEF1EF0040E495CD8B438EF23
:103BE0001EF0050E495CD8B44BEF1EF0060E495C82
:103BF000D8B459EF1EF0080E495CD8B46AEF1EF035
:103C0000FCEC41F0DFEC47F0FF0E66EC2BF0BFEC74
:103C100048F0000E66EC2BF0BFEC48F0000E66ECAE
:103C20002BF06AEF1EF071EC41F0DFEC47F0FF0E75
:103C300066EC2BF0BFEC48F0000E66EC2BF06AEF60
:103C40001EF089EC41F0DFEC47F0FF0E66EC2BF044
:103C50006AEF1EF0A6EC41F0DFEC47F0FF0E66ECD9
:103C60002BF0BFEC48F0000E66EC2BF06AEF1EF074
:103C7000BEEC41F0DFEC47F0FF0E66EC2BF0BFEC42
:103C800048F0000E66EC2BF0BFEC48F0000E66EC3E
:103C90002BF06AEF1EF0D1EC41F0DFEC47F0FF0EA5
:103CA00066EC2BF0BFEC48F0000E66EC2BF06AEFF0
:103CB0001EF0E9EC41F0DFEC47F0FF0E66EC2BF074
:103CC000BFEC48F0000E66EC2BF0BFEC48F0000EA5
:103CD00066EC2BF03FB671EF1EF03F8618504A6E2F
:103CE0004B6E97EC32F02BEC2BF0400E34EC2BF0BB
:103CF000BD0E4DEC2BF0405046EC3AF08FEC3AF014
:103D00003F82FEEF20F05FEC40F03FB28AEF1EF002
:103D1000070E496E3FA45AEC32F028EC2BF0460E09
:103D200034EC2BF0BC0E4DEC2BF0010E495CD8B4FA
:103D3000CBEF1EF0020E495CD8B4D9EF1EF0030E93
:103D4000495CD8B4E2EF1EF0040E495CD8B4F0EF41
:103D50001EF0050E495CD8B403EF1FF0060E495C57
:103D6000D8B411EF1FF0080E495CD8B422EF1FF051
:103D7000FCEC41F05FEC43F0FF0E66EC2BF0BFEC87
:103D800048F0000E66EC2BF0BFEC48F0000E66EC3D
:103D90002BF022EF1FF071EC41F05FEC43F0FF0ECF
:103DA00066EC2BF0BFEC48F0000E66EC2BF022EF37
:103DB0001FF089EC41F05FEC43F0FF0E66EC2BF056
:103DC00022EF1FF0A6EC41F05FEC43F0FF0E66EC33
:103DD0002BF0BFEC48F0000E66EC2BF022EF1FF04A
:103DE000BEEC41F05FEC43F0FF0E66EC2BF0BFEC55
:103DF00048F0000E66EC2BF0BFEC48F0000E66ECCD
:103E00002BF022EF1FF0D1EC41F05FEC43F0FF0EFE
:103E100066EC2BF0BFEC48F0000E66EC2BF022EFC6
:103E20001FF0E9EC41F05FEC43F0FF0E66EC2BF085
:103E3000BFEC48F0000E66EC2BF0BFEC48F0000E33
:103E400066EC2BF03FB629EF1FF03F8619504A6E03
:103E50004B6E97EC32F02BEC2BF0400E34EC2BF049
:103E6000BD0E4DEC2BF0405046EC3AF08FEC3AF0A2
:103E70003F82FEEF20F0E8EC40F03FB242EF1FF04F
:103E8000070E496E3FA45AEC32F028EC2BF0460E98
:103E900034EC2BF0BC0E4DEC2BF0010E495CD8B489
:103EA00083EF1FF0020E495CD8B491EF1FF0030EB0
:103EB000495CD8B49AEF1FF0040E495CD8B4A8EF5F
:103EC0001FF0050E495CD8B4BBEF1FF0060E495C2D
:103ED000D8B4C9EF1FF0080E495CD8B4DAEF1FF070
:103EE000FCEC41F04FEC43F0FF0E66EC2BF0BFEC26
:103EF00048F0000E66EC2BF0BFEC48F0000E66ECCC
:103F00002BF0DAEF1FF071EC41F04FEC43F0FF0EB5
:103F100066EC2BF0BFEC48F0000E66EC2BF0DAEF0D
:103F20001FF089EC41F04FEC43F0FF0E66EC2BF0F4
:103F3000DAEF1FF0A6EC41F04FEC43F0FF0E66EC19
:103F40002BF0BFEC48F0000E66EC2BF0DAEF1FF020
:103F5000BEEC41F04FEC43F0FF0E66EC2BF0BFECF3
:103F600048F0000E66EC2BF0BFEC48F0000E66EC5B
:103F70002BF0DAEF1FF0D1EC41F04FEC43F0FF0EE5
:103F800066EC2BF0BFEC48F0000E66EC2BF0DAEF9D
:103F90001FF0E9EC41F04FEC43F0FF0E66EC2BF024
:103FA000BFEC48F0000E66EC2BF0BFEC48F0000EC2
:103FB00066EC2BF03FB6E1EF1FF03F861A504A6ED9
:103FC0004B6E97EC32F02BEC2BF0400E34EC2BF0D8
:103FD000BD0E4DEC2BF0405046EC3AF08FEC3AF031
:103FE0003F82FEEF20F0BFEC45F0000E66EC2BF0B8
:103FF000CFEC45F0000E66EC2BF0DFEC45F0000E48
:1040000066EC2BF08FEC45F0000E66EC2BF0BFEC6D
:1040100046F0000E66EC2BF02FEC46F0000E66EC3E
:104020002BF0AFEC46F0000E66EC2BF0BFEC48F046
:104030002FEC46F0000E66EC2BF05FEC46F02BEC1C
:104040002BF0400E34EC2BF0B90E4DEC2BF0000EA3
:1040500066EC2BF08FEC45F0000E66EC2BF0BFEC1D
:1040600045F0000E66EC2BF028EC2BF0670E34ECDC
:104070002BF0BC0E4DEC2BF03FB053EF20F0000EB8
:1040800066EC2BF0FFEC46F0000E66EC2BF0CFEC6C
:1040900045F0000E66EC2BF09FEC46F0000E66EC4F
:1040A0002BF065EF20F0FF0E66EC2BF09FEC48F054
:1040B000FF0E66EC2BF05FEC47F0FF0E66EC2BF08A
:1040C0003FEC48F0FF0E66EC2BF02BEC2BF0440E8F
:1040D00034EC2BF0BC0E4DEC2BF03FB084EF20F015
:1040E000FF0E66EC2BF0EFEC47F0FF0E66EC2BF0CA
:1040F000CFEC48F0FF0E66EC2BF0FFEC47F0FF0E24
:1041000066EC2BF096EF20F0000E66EC2BF04FECF7
:1041100046F0000E66EC2BF0BFEC48F0000E66ECAB
:104120002BF05FEC46F0000E66EC2BF080B0AFEFAA
:1041300020F0070E555CD8B4A1EF20F0552AB1EF5E
:1041400020F0556A3EB0B1EF20F03FB0ABEF20F069
:104150003F80ACEF20F03F903E80B1EF20F03E90EA
:10416000556A84B6CAEF20F0070E545CD8B4BCEF91
:1041700020F0542ACCEF20F0546A3EBCCCEF20F063
:104180003FB0C6EF20F03F80C7EF20F03F903E8C5D
:10419000CCEF20F03E9C546A80B8FCEF20F0070E74
:1041A000575CD8B4D7EF20F0572AFEEF20F0576ABB
:1041B0003EB8FEEF20F0436A466A50EC2CF03FA078
:1041C000F8EF20F0080E116E040E126E4B0E136EF7
:1041D000BB0E146E9B0E156E880E166E7F0E176E3C
:1041E0007F0E186E000E196E000E1A6E6DEC2CF01C
:1041F0003F903E8823EF01F03E98576A3FB41FEF8F
:1042000021F080BA1DEF21F0070E565CD8B40CEFF8
:1042100021F0562A1FEF21F0566A3EBA23EF01F033
:10422000000E436E3E8A466A50EC2CF03F903F925F
:104230003F96496A4A6A23EF01F03E9A566A23EF95
:1042400001F028EC2BF0410E34EC2BF0B80E4DECC5
:104250002BF0700E66EC2BF0100E66EC2BF0100EAF
:1042600066EC2BF0100E66EC2BF0000E66EC2BF0DB
:10427000CFEC45F0000E66EC2BF0CFEC45F0000ED5
:1042800066EC2BF06FEC46F0000E66EC2BF08FEC3A
:1042900046F0000E66EC2BF05FEC46F0000E66EC8C
:1042A0002BF03FEC46F0000E66EC2BF0BFEC48F034
:1042B000DFEC46F0000E66EC2BF08FEC46F0000EC3
:1042C00066EC2BF00FEC46F02BEC2BF0400E34ECB0
:1042D0002BF0B80E4DEC2BF0000E66EC2BF0AFEC93
:1042E00046F0000E66EC2BF0CFEC45F0000E66ECCD
:1042F0002BF0082A320E085CD8B484EF21F0100E9F
:1043000066EC2BF079EF21F0086A700E66EC2BF06A
:10431000000E445CD8B494EF21F0010E445CD8B494
:104320003CEF25F023EF01F028EC2BF0460E34ECA7
:104330002BF0B90E4DEC2BF09FEC46F0000E66EC26
:104340002BF0CFEC45F0000E66EC2BF02FEC46F096
:10435000000E66EC2BF0CFEC45F0000E66EC2BF077
:10436000AFEC45F0000E66EC2BF0AFEC46F0000E23
:1043700066EC2BF0BFEC48F08FEC45F0000E66ECDD
:104380002BF0BFEC45F0000E66EC2BF0BFEC45F0D7
:104390002BEC2BF0400E34EC2BF0B90E4DEC2BF047
:1043A000000E66EC2BF08FEC46F0000E66EC2BF066
:1043B000CFEC45F0000E66EC2BF09FEC46F0000EC3
:1043C00066EC2BF09FEC46F0000E66EC2BF080B014
:1043D00002EF22F0070E555CD8B4F2EF21F0552A17
:1043E00004EF22F0556A3EB004EF22F00B0E475C5A
:1043F000D8B4FEEF21F0472AFFEF21F0476A3E8054
:1044000004EF22F03E90556A84B620EF22F0070EAA
:10441000545CD8B40FEF22F0542A22EF22F0546AF1
:104420003EBC22EF22F0000E475CD8B41BEF22F016
:1044300047061DEF22F00B0E476E3E8C22EF22F056
:104440003E9C546A28EC2BF04A0E34EC2BF0BB0E49
:104450004DEC2BF0000E475CD8B443EF22F0000E79
:1044600066EC2BF0AFEC42F0000E66EC2BF0AFECFC
:1044700042F0000E66EC2BF0FFEC45F0000E66EC0F
:104480002BF055EF22F0FF0E66EC2BF04FEC43F0D3
:10449000FF0E66EC2BF04FEC43F0FF0E66EC2BF0BA
:1044A0008FEC47F0FF0E66EC2BF028EC2BF0670E3C
:1044B00034EC2BF0BB0E4DEC2BF0010E475CD8B466
:1044C00076EF22F0000E66EC2BF0AFEC42F0000E1F
:1044D00066EC2BF0BFEC42F0000E66EC2BF0FFEC2C
:1044E00045F0000E66EC2BF088EF22F0FF0E66EC34
:1044F0002BF04FEC43F0FF0E66EC2BF05FEC43F03B
:10450000FF0E66EC2BF08FEC47F0FF0E66EC2BF005
:104510002BEC2BF0440E34EC2BF0BB0E4DEC2BF0BF
:10452000020E475CD8B4A9EF22F0000E66EC2BF027
:10453000AFEC42F0000E66EC2BF0CFEC42F0000E38
:1045400066EC2BF0FFEC45F0000E66EC2BF0BBEFB9
:1045500022F0FF0E66EC2BF04FEC43F0FF0E66EC02
:104560002BF06FEC43F0FF0E66EC2BF08FEC47F076
:10457000FF0E66EC2BF02BEC2BF0610E34EC2BF0E5
:10458000BB0E4DEC2BF0030E475CD8B4DCEF22F0F1
:10459000000E66EC2BF0AFEC42F0000E66EC2BF058
:1045A000DFEC42F0000E66EC2BF0FFEC45F0000E65
:1045B00066EC2BF0EEEF22F0FF0E66EC2BF04FECEA
:1045C00043F0FF0E66EC2BF07FEC43F0FF0E66EC41
:1045D0002BF08FEC47F0FF0E66EC2BF028EC2BF065
:1045E0004A0E34EC2BF0BC0E4DEC2BF0040E475C65
:1045F000D8B40FEF23F0000E66EC2BF0AFEC42F0D6
:10460000000E66EC2BF0EFEC42F0000E66EC2BF0A7
:10461000FFEC45F0000E66EC2BF021EF23F0FF0ECF
:1046200066EC2BF04FEC43F0FF0E66EC2BF08FECBA
:1046300043F0FF0E66EC2BF08FEC47F0FF0E66ECBC
:104640002BF028EC2BF0670E34EC2BF0BC0E4DEC6D
:104650002BF0050E475CD8B442EF23F0000E66EC59
:104660002BF0AFEC42F0000E66EC2BF0FFEC42F0CA
:10467000000E66EC2BF0FFEC45F0000E66EC2BF024
:1046800054EF23F0FF0E66EC2BF04FEC43F0FF0EDF
:1046900066EC2BF09FEC43F0FF0E66EC2BF08FECFA
:1046A00047F0FF0E66EC2BF02BEC2BF0440E34ECB5
:1046B0002BF0BC0E4DEC2BF0060E475CD8B475EF1A
:1046C00023F0000E66EC2BF0AFEC42F0000E66EC2F
:1046D0002BF00FEC43F0000E66EC2BF0FFEC45F0F6
:1046E000000E66EC2BF087EF23F0FF0E66EC2BF04C
:1046F0004FEC43F0FF0E66EC2BF0AFEC43F0FF0EF7
:1047000066EC2BF08FEC47F0FF0E66EC2BF02BECF9
:104710002BF0610E34EC2BF0B40E4DEC2BF0070EA9
:10472000475CD8B4A8EF23F0000E66EC2BF0AFEC9A
:1047300042F0000E66EC2BF01FEC43F0000E66EC2E
:104740002BF0FFEC45F0000E66EC2BF0BAEF23F0F7
:10475000FF0E66EC2BF04FEC43F0FF0E66EC2BF0F7
:10476000BFEC43F0FF0E66EC2BF08FEC47F0FF0E32
:1047700066EC2BF028EC2BF04A0E34EC2BF0BD0E3F
:104780004DEC2BF0080E475CD8B4DBEF23F0000EA5
:1047900066EC2BF0AFEC42F0000E66EC2BF02FEC49
:1047A00043F0000E66EC2BF0FFEC45F0000E66ECDB
:1047B0002BF0EDEF23F0FF0E66EC2BF04FEC43F007
:1047C000FF0E66EC2BF0CFEC43F0FF0E66EC2BF007
:1047D0008FEC47F0FF0E66EC2BF028EC2BF0670E09
:1047E00034EC2BF0BD0E4DEC2BF0090E475CD8B429
:1047F0000EEF24F0000E66EC2BF0AFEC42F0000E52
:1048000066EC2BF03FEC43F0000E66EC2BF0FFEC77
:1048100045F0000E66EC2BF020EF24F0FF0E66EC66
:104820002BF04FEC43F0FF0E66EC2BF0DFEC43F087
:10483000FF0E66EC2BF08FEC47F0FF0E66EC2BF0D2
:1048400028EC2BF04A0E34EC2BF0BE0E4DEC2BF086
:104850000A0E475CD8B45CEF24F0000E66EC2BF037
:104860005FEC46F0000E66EC2BF0AFEC46F0000E6D
:1048700066EC2BF0FFEC45F0000E66EC2BF0CFEC75
:1048800045F0000E66EC2BF08FEC46F0000E66EC67
:104890002BF0BFEC48F09FEC46F0000E66EC2BF0DE
:1048A000CFEC45F0000E66EC2BF0AFEC46F0000EBE
:1048B00066EC2BF089EF24F0FF0E66EC2BF0FFEC9A
:1048C00047F0FF0E66EC2BF04FEC48F0FF0E66EC65
:1048D0002BF08FEC47F0FF0E66EC2BF05FEC47F00F
:1048E000FF0E66EC2BF02FEC48F0FF0E66EC2BF081
:1048F000CFEC48F03FEC48F0FF0E66EC2BF05FEC9D
:1049000047F0FF0E66EC2BF04FEC48F0FF0E66EC24
:104910002BF028EC2BF04A0E34EC2BF0BF0E4DECB4
:104920002BF00B0E475CD8B4DCEF24F0000E66ECE5
:104930002BF08FEC45F0000E66EC2BF02FEC46F0E0
:10494000000E66EC2BF02FEC46F0000E66EC2BF020
:10495000BFEC48F08FEC46F0000E66EC2BF0CFEC8D
:1049600045F0000E66EC2BF0EFEC45F0000E66EC27
:104970002BF00FEC46F0000E66EC2BF09FEC46F0AF
:10498000000E66EC2BF02BEC2BF0400E34EC2BF0F1
:10499000BF0E4DEC2BF0AFEC46F0000E66EC2BF0AA
:1049A000CFEC45F0000E66EC2BF08FEC46F0000EDD
:1049B00066EC2BF020EF25F0FF0E66EC2BF01FECE1
:1049C00047F0FF0E66EC2BF0CFEC47F0FF0E66ECE5
:1049D0002BF0CFEC47F0FF0E66EC2BF0CFEC48F05D
:1049E0002FEC48F0FF0E66EC2BF05FEC47F0FF0E6B
:1049F00066EC2BF07FEC47F0FF0E66EC2BF09FECA3
:104A000047F0FF0E66EC2BF03FEC48F0FF0E66EC33
:104A10002BF02BEC2BF0400E34EC2BF0BF0E4DECBA
:104A20002BF04FEC48F0FF0E66EC2BF05FEC47F0FC
:104A3000FF0E66EC2BF02FEC48F0FF0E66EC2BF02F
:104A4000E9EC2EF080B838EF25F0070E575CD8B4AB
:104A50002DEF25F0572A3AEF25F0576A3EB83AEF86
:104A600025F0010E446E50EC2CF03E883AEF25F014
:104A70003E98576A23EF01F028EC2BF0460E34ECF9
:104A80002BF0B90E4DEC2BF0000E475CD8B47DEF47
:104A900025F0010E475CD8B485EF25F0020E475C87
:104AA000D8B48DEF25F0030E475CD8B495EF25F010
:104AB000040E475CD8B49DEF25F0050E475CD8B4D2
:104AC000A5EF25F0060E475CD8B4ADEF25F0070E34
:104AD000475CD8B4B5EF25F0080E475CD8B4BDEFFD
:104AE00025F0090E475CD8B4C5EF25F00A0E475CE7
:104AF000D8B4CDEF25F027EF26F0FCEC3CF02BEC02
:104B000035F0C4EC35F0B8EF26F055EC3DF02BEC69
:104B100035F0C4EC35F0B8EF26F0AEEC3DF02BEC00
:104B200035F0C4EC35F0B8EF26F007EC3EF02BEC96
:104B300035F0C4EC35F0B8EF26F060EC3EF02BEC2D
:104B400035F0C4EC35F0B8EF26F0B9EC3EF02BECC4
:104B500035F0C4EC35F0B8EF26F062EC3FF02BEC0A
:104B600035F0C4EC35F0B8EF26F0F0EC3FF02BEC6C
:104B700035F0C4EC35F0B8EF26F05FEC40F02BECEC
:104B800035F0C4EC35F0B8EF26F0E8EC40F02BEC53
:104B900035F0C4EC35F0B8EF26F0000E66EC2BF0E3
:104BA0005FEC46F0000E66EC2BF0AFEC46F0000E2A
:104BB00066EC2BF0FFEC45F0000E66EC2BF0CFEC32
:104BC00045F0000E66EC2BF08FEC46F0000E66EC24
:104BD0002BF0BFEC48F09FEC46F0000E66EC2BF09B
:104BE000CFEC45F0000E66EC2BF0AFEC46F0000E7B
:104BF00066EC2BF02BEC2BF0400E34EC2BF0B90EC6
:104C00004DEC2BF0000E66EC2BF0000E66EC2BF05A
:104C1000DFEC46F0000E66EC2BF08FEC46F0000E59
:104C200066EC2BF00FEC46F0000E66EC2BF0AFECD0
:104C300046F0000E66EC2BF0CFEC45F0000E66EC73
:104C40002BF02BEC35F0C4EC35F0B8EF26F08FEC00
:104C500045F0000E66EC2BF02FEC46F0000E66ECF3
:104C60002BF02FEC46F0000E66EC2BF0BFEC48F07A
:104C70008FEC46F0000E66EC2BF0CFEC45F0000E0A
:104C800066EC2BF0EFEC45F0000E66EC2BF00FEC31
:104C900046F0000E66EC2BF09FEC46F0000E66EC42
:104CA0002BF0AFEC46F02BEC2BF0400E34EC2BF05D
:104CB000B90E4DEC2BF0000E66EC2BF0CFEC45F06E
:104CC000000E66EC2BF08FEC46F0000E66EC2BF03D
:104CD000BFEC48F0DFEC46F0000E66EC2BF08FECFA
:104CE00046F0000E66EC2BF00FEC46F0000E66EC82
:104CF0002BF0AFEC46F0000E66EC2BF0CFEC45F05D
:104D0000000E66EC2BF02BEC35F080B8B6EF26F0F9
:104D1000070E575CD8B490EF26F0572AB8EF26F06C
:104D2000576A3EB8B8EF26F03FACAFEF26F050EC34
:104D30002CF0F7EC48F00AEC49F01DEC49F030ECAF
:104D400049F043EC49F056EC49F069EC49F07CEC51
:104D500049F08FEC49F0A2EC49F0B5EC49F0446A17
:104D6000476A3F9C3F903E8823EF01F03E98576A88
:104D700080BA23EF01F0070E565CD8B4C3EF26F0DB
:104D8000562A23EF01F0566A000E446E3E8A476AA7
:104D900050EC2CF03F9C23EF01F028EC2BF0410E5F
:104DA00034EC2BF0B80E4DEC2BF0700E66EC2BF0C3
:104DB000100E66EC2BF0100E66EC2BF0100E66EC6D
:104DC0002BF0000E66EC2BF05FEC46F0000E66EC6C
:104DD0002BF0AFEC46F0000E66EC2BF0FFEC45F04C
:104DE000000E66EC2BF0CFEC45F0000E66EC2BF0DD
:104DF0008FEC46F0000E66EC2BF0BFEC48F09FEC19
:104E000046F0000E66EC2BF0CFEC45F0000E66ECA1
:104E10002BF0AFEC46F0000E66EC2BF0AFEC46F05A
:104E20002BEC2BF0400E34EC2BF0B80E4DEC2BF0AD
:104E3000000E66EC2BF00FEC46F0000E66EC2BF04B
:104E40004FEC46F0000E66EC2BF0EFEC45F0000E58
:104E500066EC2BF0082A2C0E085CD8B435EF27F04E
:104E6000100E66EC2BF02AEF27F0086A700E66EC45
:104E70002BF028EC2BF0460E34EC2BF0BF0E4DEC53
:104E80002BF09FEC46F0000E66EC2BF05FEC46F04A
:104E9000000E66EC2BF0DFEC45F0000E66EC2BF01C
:104EA000AFEC46F0000E66EC2BF0DFEC46F0000EA7
:104EB00066EC2BF08FEC45F0000E66EC2BF08FECDF
:104EC00046F0000E66EC2BF0CFEC45F0000E66ECE1
:104ED0002BF0BFEC48F0CFEC46F02BEC2BF0400E63
:104EE00034EC2BF0BF0E4DEC2BF0000E66EC2BF0EB
:104EF000CFEC45F0000E66EC2BF08FEC46F0000E88
:104F000066EC2BF09FEC46F0000E66EC2BF00FECFD
:104F100046F0000E66EC2BF05FEC46F0000E66ECFF
:104F20002BF04FEC46F0000E66EC2BF0BFEC48F097
:104F3000000E66EC2BF0BFEC42F0000E66EC2BF09E
:104F4000000E66EC2BF0400E66EC2BF0000E66ECCB
:104F50002BF0AFEC42F0000E66EC2BF0DFEC42F0F1
:104F6000000E66EC2BF028EC2BF0450E34EC2BF009
:104F7000BA0E4DEC2BF04CBEFFEF27F0000E485C54
:104F8000D8A4FFEF27F0FF0E66EC2BF05FEC47F0A4
:104F9000FF0E66EC2BF02FEC48F0FF0E66EC2BF0CA
:104FA0002FEC48F0FF0E66EC2BF0FFEC47F0FF0E05
:104FB00066EC2BF02FEC48F0FF0E66EC2BF0CFECFC
:104FC00048F08FEC47F0FF0E66EC2BF0FFEC47F05B
:104FD000FF0E66EC2BF0CFEC47F0FF0E66EC2BF0EB
:104FE0004FEC47F02BEC2BF0400E34EC2BF0BA0ECC
:104FF0004DEC2BF0FF0E66EC2BF039EF28F0000E95
:1050000066EC2BF0CFEC45F0000E66EC2BF08FEC4D
:1050100046F0000E66EC2BF08FEC46F0000E66ECCE
:105020002BF05FEC46F0000E66EC2BF08FEC46F0B8
:10503000000E66EC2BF0BFEC48F0FFEC45F0000EE4
:1050400066EC2BF05FEC46F0000E66EC2BF02FECDC
:1050500046F0000E66EC2BF0BFEC45F02BEC2BF08D
:10506000400E34EC2BF0BA0E4DEC2BF0000E66EC3B
:105070002BF028EC2BF0450E34EC2BF0BB0E4DEC56
:105080002BF04CBE78EF28F0010E485CD8A478EFE6
:1050900028F0FF0E66EC2BF04FEC48F0FF0E66ECAC
:1050A0002BF08FEC48F0FF0E66EC2BF0CFEC48F0C5
:1050B000FFEC47F0FF0E66EC2BF05FEC48F0FF0EC4
:1050C00066EC2BF04FEC48F0FF0E66EC2BF00FEC8B
:1050D00048F0FF0E66EC2BF05FEC48F0FF0E66EC3C
:1050E0002BF04FEC48F0FF0E66EC2BF0A5EF28F00C
:1050F000000E66EC2BF0AFEC46F0000E66EC2BF0E9
:10510000EFEC46F0000E66EC2BF0BFEC48F05FECE5
:1051100046F0000E66EC2BF0BFEC46F0000E66EC9D
:105120002BF0AFEC46F0000E66EC2BF06FEC46F087
:10513000000E66EC2BF0BFEC46F0000E66EC2BF098
:10514000AFEC46F0000E66EC2BF028EC2BF0450E91
:1051500034EC2BF0BC0E4DEC2BF04CBEF1EF28F0F4
:10516000020E485CD8A4F1EF28F0FF0E66EC2BF09D
:105170003FEC48F0FF0E66EC2BF05FEC47F0FF0EC3
:1051800066EC2BF0CFEC47F0FF0E66EC2BF05FECFB
:1051900047F0FF0E66EC2BF03FEC47F0FF0E66EC9D
:1051A0002BF04FEC48F0FF0E66EC2BF0CFEC48F004
:1051B0005FEC48F0FF0E66EC2BF03FEC48F0FF0E82
:1051C00066EC2BF02FEC47F02BEC2BF0400E34EC80
:1051D0002BF0BC0E4DEC2BF0FF0E66EC2BF02BEF02
:1051E00029F0000E66EC2BF09FEC46F0000E66EC0A
:1051F0002BF0CFEC45F0000E66EC2BF02FEC46F0D8
:10520000000E66EC2BF0CFEC45F0000E66EC2BF0B8
:10521000AFEC45F0000E66EC2BF0AFEC46F0000E64
:1052200066EC2BF0BFEC48F0BFEC46F0000E66ECED
:105230002BF09FEC46F0000E66EC2BF09FEC45F057
:105240002BEC2BF0400E34EC2BF0BC0E4DEC2BF085
:10525000000E66EC2BF04CBE69EF29F080B049EFF0
:1052600029F0070E555CD8B439EF29F0552A4BEFD9
:1052700029F0556A3EB04BEF29F0020E485CD8B4D5
:1052800045EF29F0482A46EF29F0486A3E804BEF67
:1052900029F03E90556A84B667EF29F0070E545CFA
:1052A000D8B456EF29F0542A69EF29F0546A3EBC6D
:1052B00069EF29F0000E485CD8B462EF29F0480687
:1052C00064EF29F0020E486E3E8C69EF29F03E9C97
:1052D000546A4CBE83EF29F080B881EF29F0070EA5
:1052E000575CD8B477EF29F0572A83EF29F0576A33
:1052F0003EB883EF29F04C8E4C504D6E3E8883EFC4
:1053000029F03E98576A4CAE9DEF29F080BA9BEF8A
:1053100029F0070E565CD8B491EF29F0562A9DEF7C
:1053200029F0566A3EBA9DEF29F04C9E50EC2CF0C5
:105330003E8A9DEF29F03E9A566A4CAEB9EF29F0AD
:1053400080B8B7EF29F0070E575CD8B4ABEF29F05F
:10535000572AB9EF29F0576A3EB8B9EF29F04D50F6
:105360004C6E4C9E50EC2CF03E88B9EF29F03E98E4
:10537000576A4CAE14EF2AF080B0E6EF29F0070E22
:10538000555CD8B4C7EF29F0552AE8EF29F0556AE3
:105390003EB0E8EF29F0000E485CD8B4DCEF29F00D
:1053A000010E485CD8B4DFEF29F0020E485CD8B497
:1053B000E2EF29F0E3EF29F04D70E3EF29F04D72B1
:1053C000E3EF29F04D743E80E8EF29F03E90556AF6
:1053D00084B612EF2AF0070E545CD8B4F3EF29F02C
:1053E000542A14EF2AF0546A3EBC14EF2AF0000E3F
:1053F000485CD8B408EF2AF0010E485CD8B40BEF33
:105400002AF0020E485CD8B40EEF2AF00FEF2AF013
:105410004D700FEF2AF04D720FEF2AF04D743E8C55
:1054200014EF2AF03E9C546A4CAE23EF2BF0000E92
:10543000485CD8B428EF2AF0010E485CD8B465EF78
:105440002AF0020E485CD8B4D4EF2AF023EF2BF0F8
:105450002BEC2BF0460E34EC2BF0BA0E4DEC2BF06F
:105460004DA04CEF2AF0FF0E66EC2BF08FEC47F0CE
:10547000FF0E66EC2BF0FFEC47F0FF0E66EC2BF016
:10548000CFEC47F0FF0E66EC2BF04FEC47F0FF0E31
:1054900066EC2BF023EF2BF0FF0E66EC2BF06FEC9D
:1054A00047F0FF0E66EC2BF02FEC48F0FF0E66EC99
:1054B0002BF05FEC47F0FF0E66EC2BF05FEC47F053
:1054C000FF0E66EC2BF023EF2BF02BEC2BF0460EAF
:1054D00034EC2BF0BB0E4DEC2BF04DA2A2EF2AF0DA
:1054E000FF0E66EC2BF09FEC47F0FF0E66EC2BF006
:1054F000EFEC47F0FF0E66EC2BF04FEC48F0FF0EA0
:1055000066EC2BF05FEC47F0FF0E66EC2BF02FEC17
:1055100048F0FF0E66EC2BF0CFEC47F0FF0E66EC88
:105520002BF0FFEC47F0FF0E66EC2BF03FEC47F062
:10553000FF0E66EC2BF0BFEC47F0FF0E66EC2BF095
:1055400023EF2BF0FF0E66EC2BF06FEC47F0FF0E15
:1055500066EC2BF02FEC48F0FF0E66EC2BF05FECC6
:1055600047F0FF0E66EC2BF05FEC47F0FF0E66ECA9
:105570002BF0BFEC48F0000E66EC2BF0BFEC48F0CF
:10558000000E66EC2BF0BFEC48F0000E66EC2BF042
:10559000BFEC48F0000E66EC2BF0BFEC48F0000EBC
:1055A00066EC2BF023EF2BF02BEC2BF0460E34ECBB
:1055B0002BF0BC0E4DEC2BF04DA402EF2BF0FF0EA8
:1055C00066EC2BF01FEC47F0FF0E66EC2BF05FEC67
:1055D00048F0FF0E66EC2BF04FEC48F0FF0E66EC47
:1055E0002BF0FFEC47F0FF0E66EC2BF0BFEC48F021
:1055F000000E66EC2BF0BFEC48F0000E66EC2BF0D2
:1056000023EF2BF0FF0E66EC2BF0DFEC47F0FF0EE4
:1056100066EC2BF01FEC47F0FF0E66EC2BF0EFEC86
:1056200047F0FF0E66EC2BF05FEC48F0FF0E66ECE7
:105630002BF01FEC47F0FF0E66EC2BF0CFEC47F0A1
:10564000FF0E66EC2BF04CAEE9EC2EF023EF01F0F0
:105650008C888B9E12008C988B8E12008C888B8E7F
:1056600012008C988B9E1200016E2DEC2CF00150D4
:105670008A6E8C9C8C9E000000008C8A00000000CA
:105680000000000000000000000000008C9A0000F4
:1056900000000000000000001200026E2DEC2CF053
:1056A00002508A6E8C9C8C9E000000008C8A000048
:1056B00000000000000000000000000000008C9AC4
:1056C000000000000000000000001200006E2DEC41
:1056D0002CF03FBE82EC2BF000508A6E8C9C8C8E9E
:1056E000000000008C8A00000000000000000000A4
:1056F0000000000000008C9A000000000000000084
:1057000000001200000E515CD8B4A7EF2BF0010E80
:10571000515CD8B4C0EF2BF0020E515CD8B4D7EF77
:105720002BF0030E515CD8B4ECEF2BF0040E515C5F
:10573000D8B4FFEF2BF0050E515CD8B410EF2CF06D
:10574000060E515CD8B41FEF2CF02CEF2CF050B0AB
:10575000B5EF2BF0004200420042004200420042FE
:105760000042010E00162CEF2CF0004600460046C9
:105770000046004600460046800E00162CEF2CF036
:1057800050B0CDEF2BF000420042004200420042F8
:105790000042030E00162CEF2CF000460046004697
:1057A000004600460046C00E00162CEF2CF050B00C
:1057B000E3EF2BF000420042004200420042070E9D
:1057C00000162CEF2CF0004600460046004600462E
:1057D000E00E00162CEF2CF050B0F7EF2BF000424B
:1057E0000042004200420F0E00162CEF2CF0004643
:1057F000004600460046F00E00162CEF2CF050B08C
:1058000009EF2CF00042004200421F0E00162CEF60
:105810002CF0004600460046F80E00162CEF2CF047
:1058200050B019EF2CF0004200423F0E00162CEF52
:105830002CF000460046FC0E00162CEF2CF050B069
:1058400027EF2CF000427F0E00162CEF2CF00046C4
:10585000FE0E00162CEF2CF012000F01FF0E936EBF
:1058600000018C8C8C9E000000008C8A00000000DF
:105870000000000000000000000000008C9A000002
:10588000000000000000000000000000000081BED9
:1058900035EF2CF08C9C0F01000E936E000112006E
:1058A0002EEC2BF0400E34EC2BF0B80E4DEC2BF020
:1058B000000E66EC2BF0012A800E015CD8A458EF94
:1058C0002CF0022A4EEC2BF0400E34EC2BF0C00EE4
:1058D000025CD8A458EF2CF012008B8000008B9251
:1058E00078EC37F08B8278EC37F08AEC2CF0A0EC77
:1058F0002CF0B5EC2CF0CAEC2CF0DFEC2CF0F4EC36
:105900002CF009EC2DF01EEC2DF033EC2DF048ECD2
:105910002DF012008B9000005DEC2DF08B940000B8
:105920008B8600008B960000000E386E88EC2DF000
:1059300011503C6E9DEC2DF08B948B968B80120059
:105940008B905DEC2DF08B9400008B8600008B9685
:105950000000010E386E88EC2DF012503C6E9DEC6C
:105960002DF08B948B968B8012008B905DEC2DF03C
:105970008B9400008B8600008B960000020E386E20
:1059800088EC2DF013503C6E9DEC2DF08B948B9693
:105990008B8012008B905DEC2DF08B9400008B8639
:1059A00000008B960000030E386E88EC2DF014502A
:1059B0003C6E9DEC2DF08B948B968B8012008B901F
:1059C0005DEC2DF08B9400008B8600008B96000020
:1059D000040E386E88EC2DF015503C6E9DEC2DF0C9
:1059E0008B948B968B8012008B905DEC2DF08B94BA
:1059F00000008B8600008B960000050E386E88EC48
:105A00002DF016503C6E9DEC2DF08B948B968B8078
:105A100012008B905DEC2DF08B9400008B860000C3
:105A20008B960000060E386E88EC2DF017503C6EF9
:105A30009DEC2DF08B948B968B8012008B905DECFF
:105A40002DF08B9400008B8600008B960000070ED3
:105A5000386E88EC2DF018503C6E9DEC2DF08B9438
:105A60008B968B8012008B905DEC2DF08B94000058
:105A70008B8600008B960000080E386E88EC2DF0A7
:105A800019503C6E9DEC2DF08B948B968B80120000
:105A90008B905DEC2DF08B9400008B8600008B9634
:105AA0000000090E386E88EC2DF01A503C6E9DEC0B
:105AB0002DF08B948B968B8012008B9400008B863C
:105AC00000008B9600008B9400008B8600008B9664
:105AD00000008B8400008B8600008B9600008B9466
:105AE00000008B8600008B9600008B9400008B8654
:105AF00000008B9600008B9400008B8600008B9634
:105B000000008B9400008B8600008B960000120032
:105B100038BE8EEF2DF08B9490EF2DF08B8400002B
:105B20008B8600008B960000392A3846080E395CB7
:105B3000D8A488EF2DF0396A12003CBEA3EF2DF0F7
:105B40008B94A5EF2DF08B8400008B8600008B9644
:105B500000003A2A3C46080E3A5CD8A49DEF2DF08E
:105B60003A6A12008B905DEC2DF08B9400008B86CE
:105B700000008B9600000A0E386E88EC2DF08B80AA
:105B80000000000000008B905DEC2DF08B84000085
:105B90008B8600008B960000000000000000D5EC12
:105BA0002DF08B948B968B8012008B8683A0DCEF7C
:105BB0002DF03B80DDEF2DF03B903A2A8B96080EBE
:105BC0003A5CD8B4E7EF2DF03B46D5EF2DF03A6ABA
:105BD0003D2A010E3D5CD8A4F2EF2DF03B501B6E28
:105BE000D5EF2DF0020E3D5CD8A4FBEF2DF03B501D
:105BF0001C6ED5EF2DF0030E3D5CD8A404EF2EF003
:105C00003B501D6ED5EF2DF0040E3D5CD8A40DEF7A
:105C10002EF03B501E6ED5EF2DF0050E3D5CD8A446
:105C200016EF2EF03B501F6ED5EF2DF0060E3D5CAB
:105C3000D8A41FEF2EF03B50206ED5EF2DF0070EAD
:105C40003D5CD8A428EF2EF03B50216ED5EF2DF00F
:105C5000080E3D5CD8A431EF2EF03B50226ED5EFFC
:105C60002DF0090E3D5CD8A43AEF2EF03B50236E88
:105C7000D5EF2DF00A0E3D5CD8A443EF2EF03B503B
:105C8000246ED5EF2DF00B0E3D5CD8A44CEF2EF01A
:105C90003B50256ED5EF2DF00C0E3D5CD8A455EF92
:105CA0002EF03B50266ED5EF2DF00D0E3D5CD8A4A6
:105CB0005EEF2EF03B50276ED5EF2DF00E0E3D5CC3
:105CC000D8A467EF2EF03B50286ED5EF2DF00F0EC5
:105CD0003D5CD8A470EF2EF03B50296ED5EF2DF02F
:105CE000100E3D5CD8A479EF2EF03B502A6ED5EF14
:105CF0002DF0110E3D5CD8A482EF2EF03B502B6EA0
:105D0000D5EF2DF0120E3D5CD8A48BEF2EF03B505A
:105D10002C6ED5EF2DF0130E3D5CD8A494EF2EF031
:105D20003B502D6ED5EF2DF0140E3D5CD8A49DEFA9
:105D30002EF03B502E6ED5EF2DF0150E3D5CD8A405
:105D4000A6EF2EF03B502F6ED5EF2DF0160E3D5CDA
:105D5000D8A4AFEF2EF03B50306ED5EF2DF0170EDC
:105D60003D5CD8A4B8EF2EF03B50316ED5EF2DF04E
:105D7000180E3D5CD8A4C1EF2EF03B50326ED5EF2B
:105D80002DF0190E3D5CD8A4CAEF2EF03B50336EB7
:105D9000D5EF2DF01A0E3D5CD8A4D3EF2EF03B507A
:105DA000346ED5EF2DF01B0E3D5CD8A4DCEF2EF049
:105DB0003B50356ED5EF2DF01C0E3D5CD8A4E5EFC1
:105DC0002EF03B50366ED5EF2DF03B50376E3D6ACE
:105DD000120080BAFFEF2EF0070E565CD8B4F4EF35
:105DE0002EF0562A01EF2FF0566A3EBA120050EC00
:105DF0002CF0416A466A476A486A3E8A12003E9A17
:105E0000566A1200000E405CD8A42BEF2FF0EFEC86
:105E100045F0000E66EC2BF04FEC46F0000E66EC01
:105E20002BF0BFEC45F0000E66EC2BF0BFEC48F019
:105E3000000E66EC2BF0BFEC48F0000E66EC2BF089
:105E4000BFEC48F0000E66EC2BF0BFEC48F0000E03
:105E500066EC2BF01200010E405CD8A454EF2FF03A
:105E6000CFEC45F0000E66EC2BF03FEC46F0000E58
:105E700066EC2BF06FEC46F0000E66EC2BF0FFECBE
:105E800045F0000E66EC2BF0BFEC48F0000E66EC1F
:105E90002BF0BFEC48F0000E66EC2BF0BFEC48F0A6
:105EA000000E66EC2BF01200020E405CD8A47DEFD1
:105EB0002FF00FEC46F0000E66EC2BF04FEC46F0A6
:105EC000000E66EC2BF0AFEC46F0000E66EC2BF00B
:105ED000BFEC48F0000E66EC2BF0BFEC48F0000E73
:105EE00066EC2BF0BFEC48F0000E66EC2BF0BFEC3C
:105EF00048F0000E66EC2BF01200030E405CD8A4B4
:105F0000A6EF2FF0AFEC45F0000E66EC2BF0BFECE7
:105F100048F0000E66EC2BF09FEC46F0000E66ECAD
:105F20002BF0AFEC46F0000E66EC2BF08FEC45F05A
:105F3000000E66EC2BF0BFEC48F0000E66EC2BF088
:105F4000BFEC48F0000E66EC2BF01200040E405C33
:105F5000D8A4CFEF2FF0BFEC46F0000E66EC2BF08C
:105F6000BFEC48F0000E66EC2BF0BFEC45F0000EE5
:105F700066EC2BF08FEC45F0000E66EC2BF0AFECEE
:105F800046F0000E66EC2BF08FEC45F0000E66EC50
:105F90002BF0BFEC48F0000E66EC2BF01200050E63
:105FA000405CD8A4F8EF2FF08FEC46F0000E66ECC2
:105FB0002BF0BFEC48F0000E66EC2BF0CFEC45F078
:105FC000000E66EC2BF08FEC46F0000E66EC2BF02A
:105FD0008FEC46F0000E66EC2BF0BFEC48F0000EA4
:105FE00066EC2BF0BFEC48F0000E66EC2BF01200D4
:105FF000060E405CD8A421EF30F04FEC46F0000EC6
:1060000066EC2BF0CFEC46F0000E66EC2BF0BFEC0C
:1060100048F0000E66EC2BF0CFEC45F0000E66EC7D
:106020002BF08FEC46F0000E66EC2BF08FEC46F078
:10603000000E66EC2BF0BFEC48F0000E66EC2BF087
:106040001200070E405CD8A44AEF30F08FEC46F007
:10605000000E66EC2BF0AFEC45F0000E66EC2BF07A
:106060009FEC45F0000E66EC2BF02FEC46F0000E96
:1060700066EC2BF0BFEC48F0000E66EC2BF0BFECAA
:1060800048F0000E66EC2BF0BFEC48F0000E66EC1A
:106090002BF01200080E405CD8A473EF30F03FECF8
:1060A00043F0000E66EC2BF00FEC43F0000E66ECB4
:1060B0002BF01FEC46F0000E66EC2BF0FFEC45F0E9
:1060C000000E66EC2BF00FEC47F0000E66EC2BF0A8
:1060D000BFEC48F0000E66EC2BF0BFEC48F0000E71
:1060E00066EC2BF01200090E405CD8A49CEF30F057
:1060F0008FEC45F0000E66EC2BF0BFEC46F0000E86
:1061000066EC2BF0BFEC45F0000E66EC2BF00FECCC
:1061100046F0000E66EC2BF05FEC46F0000E66ECED
:106120002BF0BFEC48F0000E66EC2BF0BFEC48F013
:10613000000E66EC2BF012000A0E405CD8A4C5EFEE
:1061400030F0CFEC46F0000E66EC2BF02FEC46F072
:10615000000E66EC2BF08FEC46F0000E66EC2BF098
:10616000AFEC45F0000E66EC2BF01FEC46F0000E95
:1061700066EC2BF0BFEC48F0000E66EC2BF0BFECA9
:1061800048F0000E66EC2BF012000B0E405CD8A419
:10619000A7EF31F0AFEC46F0000E66EC2BF0EFEC21
:1061A00046F0000E66EC2BF0BFEC48F0000E66ECFB
:1061B0002BF01550070B406E000E405CD8A4F6EF94
:1061C00030F08FEC46F0000E66EC2BF0EFEC46F072
:1061D000000E66EC2BF06FEC46F0000E66EC2BF038
:1061E000AFEC42F0000E66EC2BF01200010E405CAA
:1061F000D8A410EF31F08FEC46F0000E66EC2BF0D7
:10620000EFEC46F0000E66EC2BF06FEC46F0000E63
:1062100066EC2BF0BFEC42F0000E66EC2BF01200A7
:10622000020E405CD8A42AEF31F08FEC46F0000E4D
:1062300066EC2BF0EFEC46F0000E66EC2BF06FEC0A
:1062400046F0000E66EC2BF0CFEC42F0000E66EC50
:106250002BF01200030E405CD8A444EF31F0BFECE9
:1062600046F0000E66EC2BF09FEC46F0000E66EC5C
:106270002BF09FEC45F0000E66EC2BF0BFEC48F0E5
:10628000000E66EC2BF01200040E405CD8A45EEF0A
:1062900031F08FEC46F0000E66EC2BF0EFEC46F0A0
:1062A000000E66EC2BF06FEC46F0000E66EC2BF067
:1062B000EFEC42F0000E66EC2BF01200050E405C95
:1062C000D8A478EF31F08FEC46F0000E66EC2BF09E
:1062D000EFEC46F0000E66EC2BF06FEC46F0000E93
:1062E00066EC2BF0FFEC42F0000E66EC2BF0120097
:1062F000060E405CD8A492EF31F08FEC46F0000E11
:1063000066EC2BF0EFEC46F0000E66EC2BF06FEC39
:1063100046F0000E66EC2BF00FEC43F0000E66EC3E
:106320002BF012008FEC46F0000E66EC2BF0EFEC39
:1063300046F0000E66EC2BF06FEC46F0000E66ECBB
:106340002BF01FEC43F0000E66EC2BF012000C0E4D
:10635000405CD8A4D0EF31F0CFEC46F0000E66ECF4
:106360002BF0BFEC45F0000E66EC2BF0BFEC45F0D7
:10637000000E66EC2BF0BFEC48F0000E66EC2BF044
:10638000BFEC48F0000E66EC2BF0BFEC48F0000EBE
:1063900066EC2BF0BFEC48F0000E66EC2BF0120020
:1063A0000D0E405CD8A4F9EF31F0FFEC45F0000E83
:1063B00066EC2BF08FEC46F0000E66EC2BF03FEC19
:1063C00046F0000E66EC2BF0AFEC45F0000E66ECEC
:1063D0002BF01FEC46F0000E66EC2BF0BFEC48F003
:1063E000000E66EC2BF0BFEC48F0000E66EC2BF0D4
:1063F00012008FEC46F0000E66EC2BF0CFEC45F06F
:10640000000E66EC2BF09FEC46F0000E66EC2BF0D5
:10641000CFEC45F0000E66EC2BF08FEC46F0000E52
:1064200066EC2BF0CFEC46F0000E66EC2BF0CFECD8
:1064300045F0000E66EC2BF0120080B039EF32F020
:10644000070E555CD8B428EF32F0552A3BEF32F0F6
:10645000556A3EB03BEF32F0000E495CD8A435EFF0
:1064600032F0080E496E36EF32F049063E803BEFBF
:1064700032F03E90556A84B657EF32F0070E545C06
:10648000D8B446EF32F0542A59EF32F0546A3EBC89
:1064900059EF32F0080E495CD8A453EF32F0000EE9
:1064A000496E54EF32F0492A3E8C59EF32F03E9C4F
:1064B000546A120080B076EF32F0070E555CD8B403
:1064C00065EF32F0552A78EF32F0556A3EB078EF3A
:1064D00032F0010E495CD8A472EF32F0080E496E1A
:1064E00073EF32F049063E8078EF32F03E90556A05
:1064F00084B694EF32F0070E545CD8B483EF32F0D8
:10650000542A96EF32F0546A3EBC96EF32F0080EF1
:10651000495CD8A490EF32F0010E496E91EF32F051
:10652000492A3E8C96EF32F03E9C546A1200080EC7
:10653000495CD8B4AEEF34F03FB4DDEF32F080B850
:10654000B2EF32F0070E575CD8B4AAEF32F0572AF8
:10655000B4EF32F0576A3EB870EF33F03F843E88B4
:10656000DDEF32F03E98576A28EC2BF04D0E34ECFC
:106570002BF0BE0E4DEC2BF0000E66EC2BF0BFECBA
:1065800048F0000E66EC2BF0BFEC48F0BFEC48F092
:10659000000E66EC2BF0BFEC48F0000E66EC2BF022
:1065A000BFEC48F0000E66EC2BF0BFEC48F0000E9C
:1065B00066EC2BF04A50406E120028EC2BF04D0E8A
:1065C00034EC2BF0BE0E4DEC2BF0000E495CD8B431
:1065D0000AEF33F0010E495CD8B40FEF33F0020E2E
:1065E000495CD8B414EF33F0030E495CD8B419EF0A
:1065F00033F0040E495CD8B41EEF33F0050E495C4D
:10660000D8B423EF33F0060E495CD8B428EF33F04A
:106610002DEF33F04BAE32EF33F052EF33F04BACA3
:1066200032EF33F052EF33F04BAA32EF33F052EF48
:1066300033F04BA832EF33F052EF33F04BA632EF8A
:1066400033F052EF33F04BA432EF33F052EF33F02C
:106650004BA232EF33F052EF33F04BA032EF33F076
:1066600052EF33F0000E66EC2BF0BFEC42F0000E60
:1066700066EC2BF0BFEC48F05FEC46F0000E66ECE9
:106680002BF08FEC46F0000E66EC2BF0BFEC48F0E0
:10669000FF0E66EC2BF04FEC43F0FF0E66EC2BF098
:1066A00070EF33F0FF0E66EC2BF05FEC43F0FF0E63
:1066B00066EC2BF0BFEC48F05FEC46F0000E66ECA9
:1066C0002BF08FEC46F0000E66EC2BF0BFEC48F0A0
:1066D000000E66EC2BF0AFEC42F0000E66EC2BF0F7
:1066E0004A50406E3FA4120080BA89EF33F0070E83
:1066F000565CD8B47FEF33F0562A8BEF33F0566AEE
:106700003EBA8BEF33F03F944A50406E4B6E3E8A58
:1067100012003E9A566A80B80DEF34F0070E575CAF
:10672000D8B496EF33F0572A0FEF34F0576A3EB8DB
:106730000FEF34F0000E495CD8B4BFEF33F0010E18
:10674000495CD8B4C8EF33F0020E495CD8B4D1EF3D
:1067500033F0030E495CD8B4DAEF33F0040E495C31
:10676000D8B4E3EF33F0050E495CD8B4ECEF33F066
:10677000060E495CD8B4F5EF33F0FEEF33F04BAEC4
:10678000C5EF33F04A8E07EF34F04A9E07EF34F03E
:106790004BACCEEF33F04A8C07EF34F04A9C07EF56
:1067A00034F04BAAD7EF33F04A8A07EF34F04A9A15
:1067B00007EF34F04BA8E0EF33F04A8807EF34F0EE
:1067C0004A9807EF34F04BA6E9EF33F04A8607EF1B
:1067D00034F04A9607EF34F04BA4F2EF33F04A84DA
:1067E00007EF34F04A9407EF34F04BA2FBEF33F09D
:1067F0004A8207EF34F04A9207EF34F04BA004EFDF
:1068000034F04A8007EF34F04A9007EF34F03F94B9
:106810004A50406E3E880FEF34F03E98576A80B081
:106820005CEF34F0070E555CD8B41AEF34F0552AFB
:106830005EEF34F0556A3EB05EEF34F0000E495C16
:10684000D8B443EF34F0010E495CD8B446EF34F0CD
:10685000020E495CD8B449EF34F0030E495CD8B459
:106860004CEF34F0040E495CD8B44FEF34F0050E11
:10687000495CD8B452EF34F0060E495CD8B455EFF9
:1068800034F058EF34F04B7E59EF34F04B7C59EF35
:1068900034F04B7A59EF34F04B7859EF34F04B76B3
:1068A00059EF34F04B7459EF34F04B7259EF34F028
:1068B0004B703E805EEF34F03E90556A84B6ABEF8D
:1068C00034F0070E545CD8B469EF34F0542AAEEFBC
:1068D00034F0546A3EBCADEF34F0000E495CD8B4DD
:1068E00092EF34F0010E495CD8B495EF34F0020E0B
:1068F000495CD8B498EF34F0030E495CD8B49BEFF0
:1069000034F0040E495CD8B49EEF34F0050E495CB7
:10691000D8B4A1EF34F0060E495CD8B4A4EF34F03B
:10692000A7EF34F04B7EA8EF34F04B7CA8EF34F0A7
:106930004B7AA8EF34F04B78A8EF34F04B76A8EF01
:1069400034F04B74A8EF34F04B72A8EF34F04B7076
:106950003E8CADEF34F03E9C546A120080B828EFB4
:1069600035F0070E575CD8B4B9EF34F0572A2AEF48
:1069700035F0576A3EB82AEF35F0000E465CD8B4C1
:10698000F0EF34F0010E465CD8B4F4EF34F0020EB0
:10699000465CD8B4F8EF34F0030E465CD8B4FCEF94
:1069A00034F0040E465CD8B400EF35F0050E465CBA
:1069B000D8B404EF35F0060E465CD8B408EF35F0D5
:1069C000070E465CD8B40CEF35F0080E465CD8B420
:1069D00010EF35F0090E465CD8B414EF35F0120014
:1069E0004A50116E16EF35F04A50126E16EF35F020
:1069F0004A50136E16EF35F04A50146E16EF35F00C
:106A00004A50156E16EF35F04A50166E16EF35F0F7
:106A10004A50176E16EF35F04A50186E16EF35F0E3
:106A20004A50196E16EF35F04A501A6E6DEC2CF084
:106A30004A50406E3E88000E465CD8B424EF35F0D4
:106A4000070E496E2AEF35F0050E496E2AEF35F034
:106A50003E98576A120028EC2BF0670E34EC2BF0AE
:106A6000BC0E4DEC2BF03FBC4AEF35F0000E66EC4F
:106A70002BF0FFEC46F0000E66EC2BF0CFEC45F06F
:106A8000000E66EC2BF09FEC46F0000E66EC2BF04F
:106A90005CEF35F0FF0E66EC2BF09FEC48F0FF0E3C
:106AA00066EC2BF05FEC47F0FF0E66EC2BF03FEC52
:106AB00048F0FF0E66EC2BF02BEC2BF0440E34EC80
:106AC0002BF0BC0E4DEC2BF03FBC7BEF35F0FF0EF6
:106AD00066EC2BF0EFEC47F0FF0E66EC2BF0CFEC02
:106AE00048F0FF0E66EC2BF0FFEC47F0FF0E66EC73
:106AF0002BF08DEF35F0000E66EC2BF04FEC46F0EE
:106B0000000E66EC2BF0BFEC48F0000E66EC2BF0AC
:106B10005FEC46F0000E66EC2BF080B0A6EF35F08F
:106B2000070E555CD8B498EF35F0552AA8EF35F02C
:106B3000556A3EB0A8EF35F03FBCA2EF35F03F8C70
:106B4000A3EF35F03F9C3E80A8EF35F03E90556AAC
:106B500084B6C1EF35F0070E545CD8B4B3EF35F00E
:106B6000542AC3EF35F0546A3EBCC3EF35F03FBC46
:106B7000BDEF35F03F8CBEEF35F03F9C3E8CC3EF50
:106B800035F03E9C546A120080B843EF36F0070E91
:106B9000575CD8B4CFEF35F0572A45EF36F0576A37
:106BA0003EB845EF36F03FAC3BEF36F050EC2CF002
:106BB000000E475CD8B411EF36F0010E475CD8B434
:106BC00015EF36F0020E475CD8B419EF36F0030E1D
:106BD000475CD8B41DEF36F0040E475CD8B421EF03
:106BE00036F0050E475CD8B425EF36F0060E475C4C
:106BF000D8B429EF36F0070E475CD8B42DEF36F045
:106C0000080E475CD8B431EF36F0090E475CD8B4B3
:106C100035EF36F00A0E475CD8B439EF36F03BEF6B
:106C200036F0F7EC48F03BEF36F00AEC49F03BEF7A
:106C300036F01DEC49F03BEF36F030EC49F03BEF1D
:106C400036F043EC49F03BEF36F056EC49F03BEFC1
:106C500036F069EC49F03BEF36F07CEC49F03BEF65
:106C600036F08FEC49F03BEF36F0A2EC49F03BEF09
:106C700036F0B5EC49F050EC2CF0446A476A3F9C82
:106C80003E8823EF01F03E98576A120083A266EF18
:106C900036F03FB812004CB258EF36F01550380BB2
:106CA000406E180E406E1550C70B156E60EF36F033
:106CB00015503F0B406E1B0E406E1550C00B156EED
:106CC000405015126DEC2CF03F8812003F981200D6
:106CD0001550380B406E4042404240424050070B36
:106CE000406E1550F80B156E405015121200106EC4
:106CF000000E105CD8A495EF36F005B886EF36F09C
:106D000005BA8AEF36F00FEC42F01200BFEC48F003
:106D1000058C120005BC91EF36F0059C0FEC42F09B
:106D20001200059CBFEC48F01200010E105CD8A4C4
:106D30009DEF36F01FEC42F01200020E105CD8A45A
:106D4000A5EF36F02FEC42F01200030E105CD8A431
:106D5000ADEF36F03FEC42F01200040E105CD8A408
:106D6000B5EF36F04FEC42F01200050E105CD8A4DF
:106D7000BDEF36F05FEC42F01200060E105CD8A4B6
:106D8000C5EF36F06FEC42F01200070E105CD8A48D
:106D9000CDEF36F07FEC42F01200080E105CD8A464
:106DA000D5EF36F08FEC42F012009FEC42F012006B
:106DB000106E000E105CD8A4E1EF36F0AFEC42F09C
:106DC0001200010E105CD8A4E9EF36F0BFEC42F0DF
:106DD0001200020E105CD8A4F1EF36F0CFEC42F0B6
:106DE0001200030E105CD8A4F9EF36F0DFEC42F08D
:106DF0001200040E105CD8A401EF37F0EFEC42F063
:106E00001200050E105CD8A409EF37F0FFEC42F039
:106E10001200060E105CD8A411EF37F00FEC43F00F
:106E20001200070E105CD8A419EF37F01FEC43F0E6
:106E30001200080E105CD8A421EF37F02FEC43F0BD
:106E400012003FEC43F01200106E000E105CD8A44C
:106E50002DEF37F04FEC43F01200010E105CD8A478
:106E600035EF37F05FEC43F01200020E105CD8A44F
:106E70003DEF37F06FEC43F01200030E105CD8A426
:106E800045EF37F07FEC43F01200040E105CD8A4FD
:106E90004DEF37F08FEC43F01200050E105CD8A4D4
:106EA00055EF37F09FEC43F01200060E105CD8A4AB
:106EB0005DEF37F0AFEC43F01200070E105CD8A482
:106EC00065EF37F0BFEC43F01200080E105CD8A459
:106ED0006DEF37F0CFEC43F01200DFEC43F012001F
:106EE000062A0A0E065CD8A470EF37F0066A120074
:106EF000062AFF0E065CD8A478EF37F0066A072A48
:106F0000640E075CD8A478EF37F0066A076A1200AF
:106F1000062AFF0E065CD8A488EF37F0066A072A17
:106F2000FF0E075CD8A488EF37F0066A076A1200E4
:106F300028EC2BF0400E34EC2BF0BF0E4DEC2BF078
:106F4000BFEC45F0000E66EC2BF08FEC45F0000E28
:106F500066EC2BF00FEC46F0000E66EC2BF02FECFD
:106F600043F0000E66EC2BF0EFEC42F0000E66EC06
:106F70002BF0BFEC42F0000E66EC2BF00FEC43F070
:106F8000BFEC48F08FEC46F0000E66EC2BF0CFEC37
:106F900045F0000E66EC2BF0CFEC46F02BEC2BF01E
:106FA000400E34EC2BF0BF0E4DEC2BF0400E66EC97
:106FB0002BF0000E66EC2BF0BFEC42F0000E66ECFE
:106FC0002BF0400E66EC2BF0000E66EC2BF0AFECD5
:106FD00042F0000E66EC2BF0400E036E7F0E046E46
:106FE00028EC2BF0035034EC2BF0BC0E4DEC2BF0C6
:106FF000010E66EC2BF02BEC2BF0045034EC2BF054
:10700000BC0E4DEC2BF0010E66EC2BF0032A0406AF
:1070100078EC37F0800E035CD8A4F0EF37F088EC02
:1070200037F088EC37F088EC37F088EC37F088ECF4
:1070300037F0400E036E7F0E046E28EC2BF00350E9
:1070400034EC2BF0BC0E4DEC2BF0000E66EC2BF06C
:107050002BEC2BF0045034EC2BF0BC0E4DEC2BF051
:10706000000E66EC2BF0032A040678EC37F0800E55
:10707000035CD8A41DEF38F03F8E88EC37F088EC25
:1070800037F088EC37F088EC37F0508028EC2BF0A4
:107090004A0E34EC2BF0BB0E4DEC2BF03FEC44F0E1
:1070A000000E66EC2BF0100E66EC2BF0100E66EC6A
:1070B0002BF0100E66EC2BF0100E66EC2BF0100E81
:1070C00066EC2BF0000E66EC2BF0BFEC44F0000EEB
:1070D00066EC2BF0BFEC48F0000E66EC2BF02FECCA
:1070E00044F0000E66EC2BF0BFEC44F0000E66ECB2
:1070F0002BF04FEC44F0000E66EC2BF06FEC44F0FC
:10710000000E66EC2BF0BFEC44F0000E66EC2BF0AA
:107110002BEC2BF0400E34EC2BF0BB0E4DEC2BF097
:107120002FEC44F0000E66EC2BF02FEC44F0000E38
:1071300066EC2BF0FFEC44F0000E66EC2BF06FECED
:1071400044F0000E66EC2BF0BFEC44F0000E66EC51
:107150002BF04FEC44F0000E66EC2BF0509028EC36
:107160002BF0560E34EC2BF0BC0E4DEC2BF0EFEC6C
:1071700043F0000E66EC2BF02FEC45F0000E66ECB1
:107180002BF01FEC44F0000E66EC2BF06FEC44F09B
:10719000000E66EC2BF0CFEC44F0000E66EC2BF00A
:1071A000BFEC48F0000E66EC2BF09FEC44F0000EB4
:1071B00066EC2BF02BEC2BF0400E34EC2BF0BC0EDD
:1071C0004DEC2BF0EFEC43F0000E66EC2BF0FFECF7
:1071D00043F0000E66EC2BF0CFEC44F0000E66ECB2
:1071E0002BF0FFEC44F0000E66EC2BF0EFEC43F0DC
:1071F000000E66EC2BF01FEC45F0000E66EC2BF059
:10720000CFEC44F0000E66EC2BF0FFEC44F0000EE7
:1072100066EC2BF06FEC45F0000E66EC2BF0512A7B
:10722000080E515CD8A43DEF38F03F9E516A88ECBF
:1072300037F088EC37F088EC37F088EC37F088ECE2
:1072400037F088EC37F088EC37F088EC37F088ECD2
:1072500037F088EC37F088EC37F088EC37F088ECC2
:1072600037F088EC37F088EC37F088EC37F088ECB2
:1072700037F088EC37F088EC37F088EC37F088ECA2
:1072800037F088EC37F088EC37F088EC37F088EC92
:1072900037F088EC37F088EC37F088EC37F088EC82
:1072A00037F088EC37F088EC37F088EC37F088EC72
:1072B00037F088EC37F088EC37F088EC37F088EC62
:1072C00037F088EC37F088EC37F088EC37F088EC52
:1072D00037F088EC37F088EC37F088EC37F088EC42
:1072E00037F088EC37F088EC37F088EC37F088EC32
:1072F00037F088EC37F088EC37F088EC37F088EC22
:1073000037F088EC37F088EC37F088EC37F088EC11
:1073100037F088EC37F088EC37F088EC37F088EC01
:1073200037F088EC37F088EC37F088EC37F088ECF1
:1073300037F088EC37F088EC37F088EC37F088ECE1
:1073400037F088EC37F088EC37F088EC37F088ECD1
:1073500037F088EC37F050EC2CF088EC37F088EC04
:1073600037F088EC37F088EC37F01200096E640EC5
:10737000095ED8A0BFEF39F00A2AB7EF39F0640EE2
:1073800009260A0E095ED8A0C9EF39F00B2AC1EF11
:1073900039F00A0E0926010E095ED8A0D3EF39F0A4
:1073A0000C2ACBEF39F012000D6E100E0D5ED8A036
:1073B000DDEF39F00B2AD5EF39F0100E0D26010E56
:1073C0000D5ED8A0E7EF39F00C2ADFEF39F012009C
:1073D00005880A5077EC36F0000E66EC2BF0059825
:1073E000058A0B5077EC36F0000E66EC2BF0059A10
:1073F0000C5077EC36F0000E66EC2BF00A6A0B6A44
:107400000C6A12000A50D8EC36F0000E66EC2BF035
:107410000B50D8EC36F0000E66EC2BF00C50D8EC8C
:1074200036F0000E66EC2BF00A6A0B6A0C6A12004A
:107430000A5024EC37F0FF0E66EC2BF00B5024ECD6
:1074400037F0FF0E66EC2BF00C5024EC37F0FF0EFB
:1074500066EC2BF00A6A0B6A0C6A1200406E452A31
:10746000090E455CD8B444EF3AF040BE3CEF3AF028
:10747000AFEC42F03EEF3AF0BFEC42F0000E66ECAB
:107480002BF040462FEF3AF0456A1200406E080E8E
:10749000455CD8B483EF3AF040BE68EF3AF045500F
:1074A000495CD8B45EEF3AF0000E66EC2BF0AFEC1E
:1074B00042F0000E66EC2BF07FEF3AF0FF0E66EC28
:1074C0002BF04FEC43F0FF0E66EC2BF07FEF3AF021
:1074D0004550495CD8B477EF3AF0000E66EC2BF0DB
:1074E000BFEC42F0000E66EC2BF07FEF3AF0FF0E9F
:1074F00066EC2BF05FEC43F0FF0E66EC2BF0452AB8
:10750000404647EF3AF0456A12007D0E4F5CD8B412
:107510008CEF3AF04F2A12003F8A4F6A12002BEC90
:107520002BF0530E34EC2BF0BE0E4DEC2BF0080E6E
:10753000495CD8A4E7EF3AF0FF0E66EC2BF03FEC85
:1075400048F0FF0E66EC2BF05FEC47F0FF0E66ECA8
:107550002BF04FEC48F0FF0E66EC2BF028EC2BF0F4
:10756000460E34EC2BF0BC0E4DEC2BF0000E66EC0E
:107570002BF0BFEC48F0000E66EC2BF0BFEC48F0AF
:10758000000E66EC2BF0BFEC48F0000E66EC2BF022
:10759000BFEC48F0000E66EC2BF0BFEC48F0000E9C
:1075A00066EC2BF0BFEC48F0000E66EC2BF0BFEC65
:1075B00048F0000E66EC2BF0BFEC48F0000E66ECD5
:1075C0002BF0BFEC48F0000E66EC2BF01200000E22
:1075D00066EC2BF09FEC46F0000E66EC2BF0CFEC47
:1075E00045F0000E66EC2BF0AFEC46F0000E66ECBA
:1075F0002BF012002BEC2BF0400E34EC2BF0BB0EDA
:107600004DEC2BF01200000E66EC2BF04FEC46F028
:10761000000E66EC2BF05FEC46F0000E66EC2BF0F3
:10762000BFEC48F0000E66EC2BF085EC3CF0BFECB4
:1076300048F0000E66EC2BF0BFEC48F0BFEC48F0D1
:10764000E0EC3CF01200FF0E66EC2BF01FEC48F073
:10765000FF0E66EC2BF03FEC47F0FF0E66EC2BF0D4
:107660002FEC48F0FF0E66EC2BF03FEC47F0FF0EDE
:1076700066EC2BF0CFEC48F0FF0E66EC2BF09FECA5
:107680003CF0E0EC3CF01200FF0E66EC2BF03FEC1F
:1076900047F0FF0E66EC2BF03FEC47F0FF0E66EC78
:1076A0002BF02FEC48F0FF0E66EC2BF03FEC47F090
:1076B000FF0E66EC2BF0CFEC48F0FF0E66EC2BF0E3
:1076C0009FEC3CF0E0EC3CF01200FF0E66EC2BF07F
:1076D0005FEC48F0FF0E66EC2BF0EFEC47F0FF0E8E
:1076E00066EC2BF0CFEC47F0FF0E66EC2BF0FFECD6
:1076F00047F0FF0E66EC2BF03FEC47F0FF0E66EC18
:107700002BF0BFEC47F0FF0E66EC2BF0BFEC48F01F
:10771000000E66EC2BF0BFEC48F0000E66EC2BF090
:10772000BFEC48F0000E66EC2BF0BFEC48F0000E0A
:1077300066EC2BF0E0EC3CF01200FF0E66EC2BF058
:107740006FEC48F0FF0E66EC2BF01FEC47F0FF0EDD
:1077500066EC2BF0CFEC47F0FF0E66EC2BF09FECC5
:1077600047F0FF0E66EC2BF04FEC47F0FF0E66EC97
:107770002BF09FEC47F0FF0E66EC2BF04FEC48F03F
:10778000FF0E66EC2BF09FEC48F0FF0E66EC2BF042
:10779000CFEC48F05FEC47F0FF0E66EC2BF0810E6B
:1077A00066EC2BF0ED0E66EC2BF0ED0E66EC2BF09C
:1077B000ED0E66EC2BF0FAEC3AF0930E66EC2BF043
:1077C000FF0E66EC2BF0A9EC3CF0BFEC48F0000E8D
:1077D00066EC2BF01200FF0E66EC2BF02FEC47F05E
:1077E000FF0E66EC2BF09FEC47F0FF0E66EC2BF0E3
:1077F000CFEC48F0FF0E66EC2BF00FEC48F0FF0EDC
:1078000066EC2BF08FEC47F0FF0E66EC2BF01FECD4
:1078100047F0FF0E66EC2BF03FEC48F0FF0E66ECF5
:107820002BF05FEC47F0FF0E66EC2BF0CFEC48F04E
:107830005FEC47F0FF0E66EC2BF0810E66EC2BF050
:10784000ED0E66EC2BF0ED0E66EC2BF0ED0E66EC1B
:107850002BF0FAEC3AF0930E66EC2BF0FF0E66EC90
:107860002BF0A9EC3CF0BFEC48F0000E66EC2BF0DE
:107870001200FF0E66EC2BF00FEC48F0FF0E66ECEA
:107880002BF01FEC47F0FF0E66EC2BF02FEC48F0CE
:10789000FF0E66EC2BF09FEC47F0FF0E66EC2BF032
:1078A0004FEC48F0FF0E66EC2BF09FEC48F0FF0E1B
:1078B00066EC2BF0CFEC48F05FEC47F0FF0E66EC87
:1078C0002BF02FEC48F0FF0E66EC2BF02FEC48F07D
:1078D000FF0E66EC2BF0C30E66EC2BF0BD0E66ECD3
:1078E0002BF0BD0E66EC2BF0BD0E66EC2BF0FAEC27
:1078F0003AF0C30E66EC2BF0FF0E66EC2BF0B3EC07
:107900003CF0000E66EC2BF01200CFEC45F0000EC0
:1079100066EC2BF08FEC46F0000E66EC2BF08FEC53
:1079200046F0000E66EC2BF05FEC46F0000E66ECC5
:107930002BF08FEC46F0000E66EC2BF012005FECA3
:1079400047F0FF0E66EC2BF02FEC48F0FF0E66ECD4
:107950002BF02FEC48F0FF0E66EC2BF0FFEC47F01D
:10796000FF0E66EC2BF02FEC48F0FF0E66EC2BF0D0
:1079700012009FEC3CF0CFEC48F0FF0E66EC2BF0D1
:107980003FEC47F0FF0E66EC2BF0FFEC47F0FF0EEC
:1079900066EC2BF04FEC47F0FF0E66EC2BF05FEC43
:1079A00047F0FF0E66EC2BF0FF0E66EC2BF0FF0E9F
:1079B00066EC2BF0FF0E66EC2BF0FAEC3AF01200BE
:1079C000FAEC3AF0BFEC48F0000E66EC2BF0BFEC9E
:1079D00048F0000E66EC2BF0BFEC48F0000E66ECB1
:1079E0002BF0BFEC48F0000E66EC2BF0BFEC48F03B
:1079F000000E66EC2BF01200AFEC45F0000E66ECCA
:107A00002BF05FEC46F0000E66EC2BF04FEC46F0EE
:107A1000000E66EC2BF0AFEC46F0000E66EC2BF09F
:107A20008FEC46F0000E66EC2BF05FEC46F0000E9B
:107A300066EC2BF02FEC46F0000E66EC2BF0BFEC62
:107A400048F0AFEC42F0000E66EC2BF0BFEC48F0D3
:107A50002BEC2BF0400E34EC2BF0B90E4DEC2BF050
:107A6000FF0E66EC2BF0810E66EC2BF0810E66ECBF
:107A70002BF0000E66EC2BF0AFEC42F0000E66EC43
:107A80002BF0AFEC42F0000E66EC2BF0FFEC45F073
:107A9000000E66EC2BF0810E66EC2BF0810E66EC8E
:107AA0002BF0FF0E66EC2BF01200AFEC45F0000E51
:107AB00066EC2BF05FEC46F0000E66EC2BF04FEC22
:107AC00046F0000E66EC2BF0AFEC46F0000E66ECD4
:107AD0002BF08FEC46F0000E66EC2BF05FEC46F0DE
:107AE000000E66EC2BF02FEC46F0000E66EC2BF04F
:107AF000BFEC48F0BFEC42F0000E66EC2BF0BFECA0
:107B000048F02BEC2BF0400E34EC2BF0B90E4DEC82
:107B10002BF0FF0E66EC2BF0810E66EC2BF0810E45
:107B200066EC2BF0000E66EC2BF0AFEC42F0000E92
:107B300066EC2BF0BFEC42F0000E66EC2BF0FFEC95
:107B400045F0000E66EC2BF0810E66EC2BF0810EFA
:107B500066EC2BF0FF0E66EC2BF01200AFEC45F05C
:107B6000000E66EC2BF05FEC46F0000E66EC2BF09E
:107B70004FEC46F0000E66EC2BF0AFEC46F0000E3A
:107B800066EC2BF08FEC46F0000E66EC2BF05FEC11
:107B900046F0000E66EC2BF02FEC46F0000E66EC83
:107BA0002BF0BFEC48F0CFEC42F0000E66EC2BF06F
:107BB000BFEC48F02BEC2BF0400E34EC2BF0B90E60
:107BC0004DEC2BF0FF0E66EC2BF0810E66EC2BF0EB
:107BD000810E66EC2BF0000E66EC2BF0AFEC42F061
:107BE000000E66EC2BF0CFEC42F0000E66EC2BF0B2
:107BF000FFEC45F0000E66EC2BF0810E66EC2BF0EE
:107C0000810E66EC2BF0FF0E66EC2BF01200AFEC51
:107C100045F0000E66EC2BF05FEC46F0000E66ECD3
:107C20002BF04FEC46F0000E66EC2BF0AFEC46F07C
:107C3000000E66EC2BF08FEC46F0000E66EC2BF09D
:107C40005FEC46F0000E66EC2BF02FEC46F0000ED9
:107C500066EC2BF0BFEC48F0DFEC42F0000E66EC77
:107C60002BF0BFEC48F02BEC2BF0400E34EC2BF05B
:107C7000B90E4DEC2BF0FF0E66EC2BF0810E66EC8E
:107C80002BF0810E66EC2BF0000E66EC2BF0AFECC7
:107C900042F0000E66EC2BF0DFEC42F0000E66ECDA
:107CA0002BF0FFEC45F0000E66EC2BF0810E66EC3D
:107CB0002BF0810E66EC2BF0FF0E66EC2BF0120021
:107CC000AFEC45F0000E66EC2BF05FEC46F0000EDA
:107CD00066EC2BF04FEC46F0000E66EC2BF0AFECB0
:107CE00046F0000E66EC2BF08FEC46F0000E66ECD2
:107CF0002BF05FEC46F0000E66EC2BF02FEC46F01C
:107D0000000E66EC2BF0BFEC48F0EFEC42F0000EFA
:107D100066EC2BF0BFEC48F02BEC2BF0400E34EC73
:107D20002BF0B90E4DEC2BF0FF0E66EC2BF0810E14
:107D300066EC2BF0810E66EC2BF0000E66EC2BF05F
:107D4000AFEC42F0000E66EC2BF0EFEC42F0000ED0
:107D500066EC2BF0FFEC45F0000E66EC2BF0810E8C
:107D600066EC2BF0810E66EC2BF0FF0E66EC2BF030
:107D700012009FEC46F0000E66EC2BF0CFEC45F0C5
:107D8000000E66EC2BF08FEC46F0000E66EC2BF04C
:107D90000FEC46F0000E66EC2BF08FEC45F0000E79
:107DA00066EC2BF02FEC46F0000E66EC2BF0BFECEF
:107DB00048F08FEC45F0000E66EC2BF0BFEC46F07F
:107DC000000E66EC2BF0BFEC45F02BEC2BF0400ED8
:107DD00034EC2BF0B90E4DEC2BF0000E66EC2BF0D2
:107DE0000FEC46F0000E66EC2BF05FEC46F0000E58
:107DF00066EC2BF028EC2BF04C0E34EC2BF0BA0E8A
:107E00004DEC2BF0BFEC45F0000E66EC2BF08FEC48
:107E100045F0000E66EC2BF0AFEC46F0000E66EC81
:107E20002BF08FEC45F0000E66EC2BF0BFEC48F029
:107E3000DFEC45F0000E66EC2BF05FEC46F0000E38
:107E400066EC2BF08FEC46F0000E66EC2BF03FEC6E
:107E500046F02BEC2BF0400E34EC2BF0BA0E4DEC30
:107E60002BF0000E66EC2BF08FEC45F0000E66EC6C
:107E70002BF0AFEC46F0BFEC48F0FF0E66EC2BF0B9
:107E8000810E66EC2BF0810E66EC2BF0000E66EC9A
:107E90002BF0AFEC42F0000E66EC2BF0FFEC42F062
:107EA000000E66EC2BF0FFEC45F0000E66EC2BF0BC
:107EB000810E66EC2BF0810E66EC2BF0FF0E66EC6B
:107EC0002BF012008FEC46F0000E66EC2BF0CFEC9E
:107ED00045F0000E66EC2BF0AFEC45F0000E66ECC2
:107EE0002BF0CFEC45F0000E66EC2BF00FEC46F0DB
:107EF000000E66EC2BF0CFEC46F0000E66EC2BF09B
:107F0000CFEC45F0000E66EC2BF08FEC46F0000E47
:107F100066EC2BF0BFEC48F0CFEC45F02BEC2BF0EF
:107F2000400E34EC2BF0B90E4DEC2BF0000E66EC4D
:107F30002BF08FEC46F0000E66EC2BF08FEC46F049
:107F4000000E66EC2BF05FEC46F0000E66EC2BF0BA
:107F50008FEC46F0000E66EC2BF0BFEC48F03FECE7
:107F600046F0000E66EC2BF08FEC45F0000E66EC50
:107F70002BF09FEC46F0000E66EC2BF01FEC46F069
:107F8000000E66EC2BF02BEC2BF0640E34EC2BF097
:107F9000BA0E4DEC2BF0FF0E66EC2BF0810E66EC6A
:107FA0002BF0810E66EC2BF0000E66EC2BF0AFECA4
:107FB00042F0000E66EC2BF00FEC43F0000E66EC86
:107FC0002BF0FFEC45F0000E66EC2BF0810E66EC1A
:107FD0002BF0810E66EC2BF0FF0E66EC2BF01200FE
:107FE0000FEC46F0000E66EC2BF04FEC46F0000E66
:107FF00066EC2BF0AFEC46F0000E66EC2BF0CFEC0D
:1080000045F0000E66EC2BF08FEC46F0000E66ECAF
:108010002BF08FEC46F0000E66EC2BF0BFEC46F038
:10802000000E66EC2BF06FEC46F0000E66EC2BF0C9
:10803000AFEC46F0BFEC48F02BEC2BF0400E34ECEC
:108040002BF0B90E4DEC2BF0000E66EC2BF03FEC54
:1080500046F0000E66EC2BF08FEC45F0000E66EC5F
:108060002BF09FEC46F0000E66EC2BF01FEC46F078
:10807000BFEC48F0FF0E66EC2BF0810E66EC2BF0A7
:10808000810E66EC2BF0000E66EC2BF0AFEC42F0AC
:10809000000E66EC2BF01FEC43F0000E66EC2BF0AC
:1080A000FFEC45F0000E66EC2BF0810E66EC2BF039
:1080B000810E66EC2BF0FF0E66EC2BF012000FEC3D
:1080C00046F0000E66EC2BF04FEC46F0000E66EC2E
:1080D0002BF0AFEC46F0000E66EC2BF0CFEC45F049
:1080E000000E66EC2BF08FEC46F0000E66EC2BF0E9
:1080F0008FEC46F0000E66EC2BF0BFEC46F0000E65
:1081000066EC2BF06FEC46F0000E66EC2BF0AFEC5B
:1081100046F0BFEC48F02BEC2BF0400E34EC2BF08B
:10812000B90E4DEC2BF0000E66EC2BF03FEC46F058
:10813000000E66EC2BF05FEC46F0000E66EC2BF0C8
:10814000BFEC45F0000E66EC2BF0CFEC45F0000ED6
:1081500066EC2BF0BFEC48F03FEC46F0000E66EC0E
:108160002BF09FEC46F0000E66EC2BF09FEC45F0F8
:10817000000E66EC2BF02BEC2BF0640E34EC2BF0A5
:10818000BA0E4DEC2BF0FF0E66EC2BF0810E66EC78
:108190002BF0810E66EC2BF0000E66EC2BF0AFECB2
:1081A00042F0000E66EC2BF02FEC43F0000E66EC74
:1081B0002BF0FFEC45F0000E66EC2BF0810E66EC28
:1081C0002BF0810E66EC2BF0FF0E66EC2BF012000C
:1081D0000FEC46F0000E66EC2BF04FEC46F0000E74
:1081E00066EC2BF0AFEC46F0000E66EC2BF0CFEC1B
:1081F00045F0000E66EC2BF08FEC46F0000E66ECBE
:108200002BF08FEC46F0000E66EC2BF0BFEC46F046
:10821000000E66EC2BF06FEC46F0000E66EC2BF0D7
:10822000AFEC46F0BFEC48F02BEC2BF0400E34ECFA
:108230002BF0B90E4DEC2BF0000E66EC2BF03FEC62
:1082400046F0000E66EC2BF05FEC46F0000E66EC9C
:108250002BF0BFEC45F0000E66EC2BF0CFEC45F0B8
:10826000000E66EC2BF0BFEC48F02FEC46F0000E51
:1082700066EC2BF09FEC46F0000E66EC2BF09FECCA
:1082800045F0000E66EC2BF02BEC2BF0640E34EC7A
:108290002BF0BA0E4DEC2BF0FF0E66EC2BF0810E9E
:1082A00066EC2BF0810E66EC2BF0000E66EC2BF0EA
:1082B000AFEC42F0000E66EC2BF03FEC43F0000E0A
:1082C00066EC2BF0FFEC45F0000E66EC2BF0810E17
:1082D00066EC2BF0810E66EC2BF0FF0E66EC2BF0BB
:1082E0001200FF0E66EC2BF00FEC48F0FF0E66EC70
:1082F0002BF03FEC47F0FF0E66EC2BF03FEC47F025
:10830000FF0E66EC2BF08FEC47F0FF0E66EC2BF0C7
:108310001200FF0E66EC2BF0FFEC47F0FF0E66EC50
:108320002BF03FEC48F0FF0E66EC2BF0CFEC47F063
:10833000FF0E66EC2BF09FEC47F0FF0E66EC2BF087
:108340000FEC48F0FF0E66EC2BF01200FF0E66EC0F
:108350002BF04FEC47F0FF0E66EC2BF05FEC47F094
:10836000FF0E66EC2BF04FEC48F0FF0E66EC2BF0A6
:108370003FEC47F0FF0E66EC2BF01200FF0E66ECB0
:108380002BF03FEC47F0FF0E66EC2BF03FEC47F094
:10839000FF0E66EC2BF08FEC47F0FF0E66EC2BF037
:1083A0001200FF0E66EC2BF02FEC48F0FF0E66EC8F
:1083B0002BF05FEC47F0FF0E66EC2BF02FEC48F053
:1083C000FF0E66EC2BF02FEC48F0FF0E66EC2BF066
:1083D0001200FF0E66EC2BF01FEC48F0FF0E66EC6F
:1083E0002BF03FEC47F0FF0E66EC2BF08FEC47F0E4
:1083F000FF0E66EC2BF01200FF0E66EC2BF06FEC1C
:1084000047F0FF0E66EC2BF03FEC47F0FF0E66ECFA
:108410002BF08FEC47F0FF0E66EC2BF012007C0E79
:1084200066EC2BF0820E66EC2BF0820E66EC2BF0E5
:10843000820E66EC2BF07C0E66EC2BF01200000E28
:1084400066EC2BF0840E66EC2BF0FE0E66EC2BF047
:10845000800E66EC2BF0000E66EC2BF01200E20EA4
:1084600066EC2BF0920E66EC2BF0920E66EC2BF085
:10847000920E66EC2BF08C0E66EC2BF01200440E84
:1084800066EC2BF0820E66EC2BF0920E66EC2BF075
:10849000920E66EC2BF06C0E66EC2BF01200300E98
:1084A00066EC2BF0280E66EC2BF0240E66EC2BF01D
:1084B000FE0E66EC2BF0200E66EC2BF012004E0E3A
:1084C00066EC2BF08A0E66EC2BF08A0E66EC2BF035
:1084D0008A0E66EC2BF0720E66EC2BF012007C0E0E
:1084E00066EC2BF0920E66EC2BF0920E66EC2BF005
:1084F000920E66EC2BF0640E66EC2BF01200060E6A
:1085000066EC2BF0020E66EC2BF0C20E66EC2BF044
:10851000320E66EC2BF00E0E66EC2BF012006C0E99
:1085200066EC2BF0920E66EC2BF0920E66EC2BF0C4
:10853000920E66EC2BF06C0E66EC2BF012004C0EDB
:1085400066EC2BF0920E66EC2BF0920E66EC2BF0A4
:10855000920E66EC2BF07C0E66EC2BF012003C0EBB
:1085600066EC2BF0420E66EC2BF0420E66EC2BF024
:10857000420E66EC2BF03C0E66EC2BF01200000E67
:1085800066EC2BF0440E66EC2BF07E0E66EC2BF0C6
:10859000400E66EC2BF0000E66EC2BF01200720E13
:1085A00066EC2BF04A0E66EC2BF04A0E66EC2BF0D4
:1085B0004A0E66EC2BF0440E66EC2BF01200220EF5
:1085C00066EC2BF04A0E66EC2BF04A0E66EC2BF0B4
:1085D0004A0E66EC2BF0340E66EC2BF01200300ED7
:1085E00066EC2BF0280E66EC2BF0240E66EC2BF0DC
:1085F0007E0E66EC2BF0200E66EC2BF012002E0E99
:1086000066EC2BF04A0E66EC2BF04A0E66EC2BF073
:108610004A0E66EC2BF0320E66EC2BF012003C0E8C
:1086200066EC2BF04A0E66EC2BF04A0E66EC2BF053
:108630004A0E66EC2BF0300E66EC2BF01200060EA4
:1086400066EC2BF0020E66EC2BF0620E66EC2BF063
:10865000120E66EC2BF00E0E66EC2BF01200340EB0
:1086600066EC2BF04A0E66EC2BF04A0E66EC2BF013
:108670004A0E66EC2BF0340E66EC2BF012000C0E5A
:1086800066EC2BF0520E66EC2BF0520E66EC2BF0E3
:10869000520E66EC2BF03C0E66EC2BF01200C30E73
:1086A00066EC2BF0BD0E66EC2BF0BD0E66EC2BF0ED
:1086B000BD0E66EC2BF0C30E66EC2BF01200FF0E25
:1086C00066EC2BF0BB0E66EC2BF0810E66EC2BF00B
:1086D000BF0E66EC2BF0FF0E66EC2BF012008D0E39
:1086E00066EC2BF0B50E66EC2BF0B50E66EC2BF0BD
:1086F000B50E66EC2BF0BB0E66EC2BF01200DD0E17
:1087000066EC2BF0B50E66EC2BF0B50E66EC2BF09C
:10871000B50E66EC2BF0CB0E66EC2BF01200CF0EF4
:1087200066EC2BF0D70E66EC2BF0DB0E66EC2BF034
:10873000810E66EC2BF0DF0E66EC2BF01200D10EF2
:1087400066EC2BF0B50E66EC2BF0B50E66EC2BF05C
:10875000B50E66EC2BF0CD0E66EC2BF01200C30EBE
:1087600066EC2BF0B50E66EC2BF0B50E66EC2BF03C
:10877000B50E66EC2BF0CF0E66EC2BF01200F90E66
:1087800066EC2BF0FD0E66EC2BF09D0E66EC2BF0EC
:10879000ED0E66EC2BF0F10E66EC2BF01200CB0E1A
:1087A00066EC2BF0B50E66EC2BF0B50E66EC2BF0FC
:1087B000B50E66EC2BF0CB0E66EC2BF01200F30E30
:1087C00066EC2BF0AD0E66EC2BF0AD0E66EC2BF0EC
:1087D000AD0E66EC2BF0C30E66EC2BF01200F80E1B
:1087E00066EC2BF0240E66EC2BF0220E66EC2BF0E0
:1087F000240E66EC2BF0F80E66EC2BF01200FE0E49
:1088000066EC2BF0920E66EC2BF0920E66EC2BF0E1
:10881000920E66EC2BF06C0E66EC2BF012007C0EC8
:1088200066EC2BF0820E66EC2BF0820E66EC2BF0E1
:10883000820E66EC2BF0440E66EC2BF01200FE0E5E
:1088400066EC2BF0820E66EC2BF0820E66EC2BF0C1
:10885000820E66EC2BF07C0E66EC2BF01200FE0E06
:1088600066EC2BF0920E66EC2BF0920E66EC2BF081
:10887000920E66EC2BF0820E66EC2BF01200FE0ED0
:1088800066EC2BF0120E66EC2BF0120E66EC2BF061
:10889000120E66EC2BF0020E66EC2BF012007C0E32
:1088A00066EC2BF0820E66EC2BF0820E66EC2BF061
:1088B000920E66EC2BF0740E66EC2BF01200FE0E9E
:1088C00066EC2BF0100E66EC2BF0100E66EC2BF025
:1088D000100E66EC2BF0FE0E66EC2BF01200000E74
:1088E00066EC2BF0820E66EC2BF0FE0E66EC2BF0A5
:1088F000820E66EC2BF0000E66EC2BF01200600E80
:1089000066EC2BF0800E66EC2BF0800E66EC2BF004
:10891000800E66EC2BF07E0E66EC2BF01200FE0E45
:1089200066EC2BF0100E66EC2BF0280E66EC2BF0AC
:10893000440E66EC2BF0820E66EC2BF01200FE0E5D
:1089400066EC2BF0800E66EC2BF0800E66EC2BF0C4
:10895000800E66EC2BF0800E66EC2BF01200FE0E03
:1089600066EC2BF0040E66EC2BF0080E66EC2BF098
:10897000040E66EC2BF0FE0E66EC2BF01200FE0EE1
:1089800066EC2BF0080E66EC2BF0100E66EC2BF06C
:10899000200E66EC2BF0FE0E66EC2BF012007C0E27
:1089A00066EC2BF0820E66EC2BF0820E66EC2BF060
:1089B000820E66EC2BF07C0E66EC2BF01200FE0EA5
:1089C00066EC2BF0120E66EC2BF0120E66EC2BF020
:1089D000120E66EC2BF00C0E66EC2BF012007C0EE7
:1089E00066EC2BF0820E66EC2BF0A20E66EC2BF000
:1089F000420E66EC2BF0BC0E66EC2BF01200FE0E65
:108A000066EC2BF0120E66EC2BF0120E66EC2BF0DF
:108A1000120E66EC2BF0EC0E66EC2BF012004C0EF6
:108A200066EC2BF0920E66EC2BF0920E66EC2BF0BF
:108A3000920E66EC2BF0640E66EC2BF01200020E28
:108A400066EC2BF0020E66EC2BF0FE0E66EC2BF0C3
:108A5000020E66EC2BF0020E66EC2BF012007E0E7E
:108A600066EC2BF0800E66EC2BF0800E66EC2BF0A3
:108A7000800E66EC2BF07E0E66EC2BF012000E0ED4
:108A800066EC2BF0300E66EC2BF0C00E66EC2BF093
:108A9000300E66EC2BF00E0E66EC2BF012001E0E64
:108AA00066EC2BF0E00E66EC2BF0180E66EC2BF06B
:108AB000E00E66EC2BF01E0E66EC2BF01200C60EDC
:108AC00066EC2BF0280E66EC2BF0100E66EC2BF00B
:108AD000280E66EC2BF0C60E66EC2BF012000E0E84
:108AE00066EC2BF0100E66EC2BF0E00E66EC2BF033
:108AF000100E66EC2BF00E0E66EC2BF01200C20E80
:108B000066EC2BF0A20E66EC2BF0920E66EC2BF0CE
:108B10008A0E66EC2BF0860E66EC2BF01200780EB7
:108B200066EC2BF0140E66EC2BF0120E66EC2BF0BC
:108B3000140E66EC2BF0780E66EC2BF012007E0E15
:108B400066EC2BF04A0E66EC2BF04A0E66EC2BF02E
:108B50004A0E66EC2BF0340E66EC2BF012003C0E45
:108B600066EC2BF0420E66EC2BF0420E66EC2BF01E
:108B7000420E66EC2BF0240E66EC2BF012007E0EFB
:108B800066EC2BF0420E66EC2BF0420E66EC2BF0FE
:108B9000420E66EC2BF03C0E66EC2BF012007E0EC3
:108BA00066EC2BF04A0E66EC2BF04A0E66EC2BF0CE
:108BB0004A0E66EC2BF0420E66EC2BF012007E0E95
:108BC00066EC2BF00A0E66EC2BF00A0E66EC2BF02E
:108BD0000A0E66EC2BF0020E66EC2BF012003C0E37
:108BE00066EC2BF0420E66EC2BF0420E66EC2BF09E
:108BF000520E66EC2BF0340E66EC2BF012007E0E5B
:108C000066EC2BF0080E66EC2BF0080E66EC2BF0F1
:108C1000080E66EC2BF07E0E66EC2BF01200000EB8
:108C200066EC2BF0420E66EC2BF07E0E66EC2BF021
:108C3000420E66EC2BF0000E66EC2BF012007E0E5E
:108C400066EC2BF0100E66EC2BF0080E66EC2BF0A9
:108C5000140E66EC2BF0620E66EC2BF012007E0E0A
:108C600066EC2BF0400E66EC2BF0400E66EC2BF021
:108C7000400E66EC2BF0400E66EC2BF012007E0EE0
:108C800066EC2BF0040E66EC2BF0080E66EC2BF075
:108C9000040E66EC2BF07E0E66EC2BF012007E0EBE
:108CA00066EC2BF0040E66EC2BF0180E66EC2BF045
:108CB000200E66EC2BF07E0E66EC2BF012003C0EC4
:108CC00066EC2BF0420E66EC2BF0420E66EC2BF0BD
:108CD000420E66EC2BF03C0E66EC2BF012007E0E82
:108CE00066EC2BF0120E66EC2BF0120E66EC2BF0FD
:108CF000120E66EC2BF00C0E66EC2BF012003C0E04
:108D000066EC2BF0420E66EC2BF0520E66EC2BF06C
:108D1000220E66EC2BF05C0E66EC2BF012007E0E41
:108D200066EC2BF0120E66EC2BF0120E66EC2BF0BC
:108D3000120E66EC2BF06C0E66EC2BF01200440E5B
:108D400066EC2BF04A0E66EC2BF04A0E66EC2BF02C
:108D50004A0E66EC2BF0320E66EC2BF01200020E7F
:108D600066EC2BF0020E66EC2BF07E0E66EC2BF020
:108D7000020E66EC2BF0020E66EC2BF012003E0E9B
:108D800066EC2BF0400E66EC2BF0400E66EC2BF000
:108D9000400E66EC2BF03E0E66EC2BF01200060E39
:108DA00066EC2BF0180E66EC2BF0600E66EC2BF0E8
:108DB000180E66EC2BF0060E66EC2BF012007E0E01
:108DC00066EC2BF0200E66EC2BF0100E66EC2BF010
:108DD000200E66EC2BF07E0E66EC2BF01200460E99
:108DE00066EC2BF0280E66EC2BF0100E66EC2BF0E8
:108DF000280E66EC2BF0460E66EC2BF01200060EE9
:108E000066EC2BF0080E66EC2BF0700E66EC2BF087
:108E1000080E66EC2BF0060E66EC2BF01200440EEA
:108E200066EC2BF0640E66EC2BF0540E66EC2BF027
:108E30004C0E66EC2BF0440E66EC2BF01200870E05
:108E400066EC2BF0EB0E66EC2BF0ED0E66EC2BF0E7
:108E5000EB0E66EC2BF0870E66EC2BF01200810E09
:108E600066EC2BF0B50E66EC2BF0B50E66EC2BF035
:108E7000B50E66EC2BF0CB0E66EC2BF01200C30E99
:108E800066EC2BF0BD0E66EC2BF0BD0E66EC2BF005
:108E9000BD0E66EC2BF0DB0E66EC2BF01200810EA3
:108EA00066EC2BF0BD0E66EC2BF0BD0E66EC2BF0E5
:108EB000BD0E66EC2BF0C30E66EC2BF01200810E9B
:108EC00066EC2BF0B50E66EC2BF0B50E66EC2BF0D5
:108ED000B50E66EC2BF0BD0E66EC2BF01200810E89
:108EE00066EC2BF0F50E66EC2BF0F50E66EC2BF035
:108EF000F50E66EC2BF0FD0E66EC2BF01200C30EA7
:108F000066EC2BF0BD0E66EC2BF0BD0E66EC2BF084
:108F1000AD0E66EC2BF0CB0E66EC2BF01200810E42
:108F200066EC2BF0F70E66EC2BF0F70E66EC2BF0F0
:108F3000F70E66EC2BF0810E66EC2BF01200FF0EA4
:108F400066EC2BF0BD0E66EC2BF0810E66EC2BF080
:108F5000BD0E66EC2BF0FF0E66EC2BF01200CF0E70
:108F600066EC2BF0BF0E66EC2BF0BF0E66EC2BF020
:108F7000BF0E66EC2BF0C10E66EC2BF01200810EDA
:108F800066EC2BF0EF0E66EC2BF0F70E66EC2BF098
:108F9000EB0E66EC2BF09D0E66EC2BF01200810EB2
:108FA00066EC2BF0BF0E66EC2BF0BF0E66EC2BF0E0
:108FB000BF0E66EC2BF0BF0E66EC2BF01200810E9C
:108FC00066EC2BF0FB0E66EC2BF0F70E66EC2BF04C
:108FD000FB0E66EC2BF0810E66EC2BF01200810E7E
:108FE00066EC2BF0FB0E66EC2BF0E70E66EC2BF03C
:108FF000DF0E66EC2BF0810E66EC2BF01200C30E38
:1090000066EC2BF0BD0E66EC2BF0BD0E66EC2BF083
:10901000BD0E66EC2BF0C30E66EC2BF01200810E39
:1090200066EC2BF0ED0E66EC2BF0ED0E66EC2BF003
:10903000ED0E66EC2BF0F30E66EC2BF01200C30E77
:1090400066EC2BF0BD0E66EC2BF0AD0E66EC2BF053
:10905000DD0E66EC2BF0A30E66EC2BF01200810EF9
:1090600066EC2BF0ED0E66EC2BF0ED0E66EC2BF0C3
:10907000ED0E66EC2BF0930E66EC2BF01200BB0E9F
:1090800066EC2BF0B50E66EC2BF0B50E66EC2BF013
:10909000B50E66EC2BF0CD0E66EC2BF01200FD0E3B
:1090A00066EC2BF0FD0E66EC2BF0810E66EC2BF0DF
:1090B000FD0E66EC2BF0FD0E66EC2BF01200C10EDF
:1090C00066EC2BF0BF0E66EC2BF0BF0E66EC2BF0BF
:1090D000BF0E66EC2BF0C10E66EC2BF01200F90E01
:1090E00066EC2BF0E70E66EC2BF09F0E66EC2BF097
:1090F000E70E66EC2BF0F90E66EC2BF01200810EF9
:1091000066EC2BF0DF0E66EC2BF0EF0E66EC2BF02E
:10911000DF0E66EC2BF0810E66EC2BF01200B90E20
:1091200066EC2BF0D70E66EC2BF0EF0E66EC2BF016
:10913000D70E66EC2BF0B90E66EC2BF01200F90E90
:1091400066EC2BF0F70E66EC2BF08F0E66EC2BF036
:10915000F70E66EC2BF0F90E66EC2BF01200000E09
:1091600066EC2BF0000E66EC2BF0040E66EC2BF098
:109170000A0E66EC2BF0040E66EC2BF01200000ECB
:1091800066EC2BF0000E66EC2BF0000E66EC2BF07C
:10919000000E66EC2BF0000E66EC2BF01200FF0EBA
:1091A00066EC2BF0FF0E66EC2BF0FF0E66EC2BF05E
:1091B000FF0E66EC2BF0FF0E66EC2BF01200280E73
:1091C00066EC2BF01200FE0E66EC2BF0FE0E66EC49
:1091D0002BF0000E66EC2BF01200000E66EC2BF06C
:1091E000000E66EC2BF0000E66EC2BF01200000E69
:1091F000AA6E000EA96E1150A86EA69EA69CA6840B
:10920000550EA76EAA0EA76EA682A6B205EF49F06C
:10921000A6941200000EAA6E010EA96E1250A86E3E
:10922000A69EA69CA684550EA76EAA0EA76EA68221
:10923000A6B218EF49F0A6941200000EAA6E020E14
:10924000A96E1350A86EA69EA69CA684550EA76E66
:10925000AA0EA76EA682A6B22BEF49F0A694120022
:10926000000EAA6E030EA96E1450A86EA69EA69CB0
:10927000A684550EA76EAA0EA76EA682A6B23EEFD2
:1092800049F0A6941200000EAA6E040EA96E1550A5
:10929000A86EA69EA69CA684550EA76EAA0EA76EC3
:1092A000A682A6B251EF49F0A6941200000EAA6E53
:1092B000050EA96E1650A86EA69EA69CA684550EF5
:1092C000A76EAA0EA76EA682A6B264EF49F0A69476
:1092D0001200000EAA6E060EA96E1750A86EA69E6A
:1092E000A69CA684550EA76EAA0EA76EA682A6B24D
:1092F00077EF49F0A6941200000EAA6E070EA96E31
:109300001850A86EA69EA69CA684550EA76EAA0EFF
:10931000A76EA682A6B28AEF49F0A6941200000EAC
:10932000AA6E080EA96E1950A86EA69EA69CA684C9
:10933000550EA76EAA0EA76EA682A6B29DEF49F0A3
:10934000A6941200000EAA6E090EA96E1A50A86EFD
:10935000A69EA69CA684550EA76EAA0EA76EA682F0
:10936000A6B2B0EF49F0A6941200000EAA6E0A0E43
:10937000A96E4C9E4C50A86EA69EA69CA684550E27
:10938000A76EAA0EA76EA682A6B2C4EF49F0A69455
:029390001200C9
:020000040030CA
:03000100331800B1
:02000500358044
:060008000FC00FE00F40E5
:0200000400F00A
:0C00000008044BBB9B887F7F00000000C1
:00000001FF
